:020000041100E9
:103000000023F7B52E4D2F4C280063616374022610
:1030100001F076F94021FE22217428002A4B009607
:1030200001F0C0F900283AD1217CFF222800274B6B
:10303000009601F0B7F9002831D1254BA2899A42B8
:103040002AD1E389234A934211D1234B6361234B55
:103050002268002A07D1002B05D019002200C1C91F
:10306000C1C21B7B6374280001F088F9F7BD1C4ABC
:10307000934201D00023EBE71A4B1B4A1B68934293
:1030800006D9C02304222800217C9B0001F000FA0D
:10309000164B6361164BDBE700232374EAE7CC236E
:1030A0003821AC2228009B01217401F0F1F900289D
:1030B000F2D1104B6361104BE381104BC8E7C0465F
:1030C000D441FF1FA861FF1FB461FF1FB661FF1F3E
:1030D000595900008305000031410011ACBD0011B9
:1030E00082150000CC61FF1F87130000E54100112D
:1030F000BCBD00117D410011AAAAFFFF9CBD0011BB
:10310000F7B5164B0192C318021D002000938823C7
:103110005B05D3181B685C1C1AD09CB2402C18D8D5
:103120008D781E0CAC466746CD782D023D43AE42ED
:1031300006D1019800280ED110000C70240A4C70A2
:1031400003249BB20733A343D218009B9A42DED3D9
:10315000FEBD4432F9E71000FAE7C046FC0F00005C
:10316000802213B503000324019189B25201073173
:103170009B18A14304305A1A88235B05C3181B68A7
:10318000591C03D190429241104016BD99B240297A
:1031900007D80B000733A343C0189042ECD300209C
:1031A000F3E74430F9E7134B134A1B68126810B574
:1031B000FA24934201D81A00F824104BE4021B6849
:1031C0009A4210D813000E4A12689A420ED3013365
:1031D00007D1F823DB029C4203D10A49054808F0D5
:1031E000EFFA200010BDFC24E402ECE7FE24E40228
:1031F000F7E7C04600C0071100D0071100E0071133
:1032000000F00711FFFFFF7FF0B59BB015000490A1
:103210000391402A00D9A0E006AB59801A80FFF73D
:10322000C2FF0400042816D9002206A9FFF768FF90
:10323000052810D906AB1B88AB420CD1002D07D056
:10324000514B2A000499C01808F07AFB002802D1DB
:1032500001201BB0F0BD06AB1D8020000699FFF7D2
:103260007FFF041E7BD1069B0793FFF79CFF802303
:103270005B01C618802307001B039E4201D3F8267A
:10328000F60288235B05F31801931B68013302D013
:10329000019808F0F5FB3D49019808F091FA3B1DB3
:1032A0000293331D05938822029B52059B181B68CD
:1032B00008935A1C3CD044219AB20091402A04D869
:1032C0000320D11D814389B2009103991B0C8B42CD
:1032D00024D0402A22D80122300008A9FFF710FF8D
:1032E000021E1BD1380008A9FFF70AFF04000428BA
:1032F00031D9009A059B9B1880225201B218934243
:1033000040D288235B05C118009A09A808F060FC28
:103310001D4B009A09A9F01808F08AFC009A029B3C
:103320009446634402931A4B029AFB189A42BAD30A
:1033300088235B05FC1821680198013908F040FAE0
:10334000200008F09DFB039A07AB5A8030000799D4
:10335000FFF706FF0400002C03D1002079E70428C2
:10336000FBD988235B05E018069908F029FA0323A6
:10337000EA1C9A4300D16BE7034B0499E01808F06C
:1033800057FC65E70424ECE704000011FFFFFF7F12
:10339000F80F0000F7B505001400402A21D80027D7
:1033A00001AE71803780FFF7FEFE042816D93A007F
:1033B0003100FFF7A5FE042810D93688BC420BD097
:1033C000BD4209D0221CB44200D9321C064B92B235
:1033D000C118280008F0FCFB30B2FEBDC04300B2AB
:1033E000FBE703204042F8E70400001137B5042250
:1033F00004000D0001A81649FFF7CCFF02000428C5
:103400000BD1019BA34208D3AB4204D0104901A8C1
:103410000195FFF7F9FE01203EBD0E4C2368200008
:10342000019308F02DFB019920000139019108F06A
:10343000C7F980235B01E418074B9C42EED10422BC
:10344000034901A80195FFF7DFFE0020E4E7C0462D
:103450005555000000C007110000081130B589B0B3
:1034600008F006F910226946254808F041FA254B74
:10347000009A9A420ED1019B029A0F2B33D8002159
:1034800001240698013B08D2002900D00292029B39
:10349000013331D10023029325E0551CF2D1020003
:1034A0002100EFE710341022200004A908F020FAD0
:1034B000029B013301D1069B0293882304995B058B
:1034C000C918059B06981A03120B049105928142B4
:1034D00003D02B4201D108F07BFB019B013B019300
:1034E000019B002BDED1029B002B03D00493049898
:1034F0004168084709B030BDE025014C2D03EFE7D6
:1035000000000111504859368022F8B5964C974B6F
:10351000D200002120001C6008F0AAFB2300944A7E
:1035200088331A60934B1A786A23002A00D011332B
:10353000E3620A232365904B37221B780820A3639C
:103540008E4B2118E361102323628D4B3B25636171
:10355000C823DB00A36123008C331A602823013ABF
:10356000E26320646364CA67043A211DCA672100CC
:10357000BC310D602100C03108602100C4310B60F6
:1035800021000635CC310D602100083DC8310D60A9
:103590002100D0310A602200D43210602200D832DB
:1035A000136022000227E032210017604222DC3142
:1035B0000A6021001B3DE4310D602100E831086004
:1035C0002100EC310B6023000521F4331960230046
:1035D000F0331A602300183290331A6023009433BA
:1035E000186023001E3A98331A60AF23DB00236073
:1035F000644BFA262363644B644DE360644BF03103
:10360000A3642300FF31FC33B600A16021611E607A
:10361000A5627325E5656D3D6565A56596255D4AE1
:10362000AD00E264666258606766A56600270925FA
:10363000A767E566584F594D606720002567E26728
:103640003A6015279C30676007001A203860200018
:10365000A0300700212038602000A83007004C4827
:1036600038602000F830066026006427A4363760F2
:1036700026005F3FAC3637602600033FB036376028
:103680002600C637B436376026000027B8363760C4
:1036900038269E60424E96205E64424E5A66DE6137
:1036A000414E9A645E62F53EFF3E9E621E269A6718
:1036B000354A8000DE661F675F67DD651D6618623C
:1036C000DA67BE23394A5B00E250394BD8382350C1
:1036D00004302250C4225200A350C623E4205B00D1
:1036E000E1500433334AE1503349344BD16034491B
:1036F000800019503349E938FF38195032490430F5
:10370000195032493248D16132491163324951630B
:103710001900F4310860CE20304940001160304972
:10372000195019002F48F83108602F49D1658221BE
:103730002E4A89005A501A002D490832D1671A00C2
:103740002C49B432116088212B4A89005A501A0042
:103750002A49883211602A4ADA6408F069F901209E
:1037600008F016F9F8BDC0460004FF1F4464FF1FAF
:10377000106FFF1F1844FF1F4A0AFF1F3A0700007F
:1037800080C3C9019A020000DC0500006A1800002D
:1037900050C3000088130000F009FF1F204E0000F6
:1037A0006509FF1F68100000C409000040420F00B7
:1037B00010270000FC00FF1F751CFF1F0000FF1FEB
:1037C000C92CFF1F5130FF1FE92EFF1F3520FF1F9F
:1037D0002527FF1F5120FF1FFD21FF1FC11FFF1FB6
:1037E0004929FF1F312AFF1F8D19FF1F5528FF1F71
:1037F0007925FF1F8525FF1FC11EFF1F791FFF1F92
:10380000391EFF1F0223F0B50124624D624E2B705A
:10381000624B91B01C70624F039333680021082003
:10382000FB7006F01FFE082006F016FD00239842EC
:1038300005D0FA78552A02D0332A00D09DE03360B3
:10384000042006F089FF07F0B3FFFFF75DFE08F0E4
:1038500017F81F2201240021524B10AE1A70524B50
:103860001C70524B1970524B19689143163A0A4317
:103870001A60602219689143403A0A431A6008F0BE
:1038800077F908F045F84B4B9847C120FF214A4B88
:1038900080001A588A431A50C522920098588843CB
:1038A000BF39014399509858444908408021C901C3
:1038B0000143802099509958C0050902090A014323
:1038C000995080213E48490108F032F80323220034
:1038D0003C49019400933C4808F0A2F92C223B4952
:1038E00005A808F075F905AC61782078023406F077
:1038F000D3FCA642F8D1364C0020012106F0E0FDB1
:103900002268344B03201A40A023DB0213432360B8
:10391000802322689B041343236022682E4B1A40A5
:1039200080239B03134323602C4A2D4B934200D8E2
:10393000012008F06DF807F093FE80232268DB0475
:1039400013432360287808F0F3F8039B1878C0B27B
:1039500007F016FF07F0BCFF2249042008F0A8F882
:1039600006F0C6FE00F040F800F0E8FD00F090FE22
:1039700000F00CFA002011B0F0BD00932100194AAC
:10398000042007F065FF8023DB059C62FFF766FDDE
:1039900056E7C0464A0AFF1F34F000401844FF1F94
:1039A000D861FF1F480AFF1F490AFF1F680AFF1F4F
:1039B000BCF00040E1A2000000E100E0FF00FFFFDA
:1039C0001C44FF1FA056FF1F1C54FF1FC0BC00114A
:1039D00014F00040FF7FF8FFFFFF9FFF0080FF1FF4
:1039E000106FFF1F3B000108002210B511001120CD
:1039F00007F03EFF10BD0000F8B500230926374F41
:103A0000374C3B62E3681120B343E36008F050F9A0
:103A1000112008F01DF8112007F0EAFF402322686A
:103A200080251343236080236268DB0213436360B5
:103A3000A3682C4A2B43A360A36802211340A36010
:103A40008023A2689B0113431022A360236C0720EC
:103A500093432364236C0F3A1343236480235B0056
:103A60003B62226B204B1A402263626B1A406263F6
:103A7000A26B1A40A263E26B1340E363E3681B4A44
:103A80001340E36006F008FC0121072006F018FD52
:103A9000174B11205A6C15435D6407F021FEFD2180
:103AA000144B154A89005A508023C720626B5B0370
:103AB00013436363E36880003343E3600F4B104AB2
:103AC00019581140802212020A431A50802292058E
:103AD0001A6008220B4B5A63F8BDC04600F0004044
:103AE0003CF00040FFFFDFFFEFFFEFFFFFFF7FFF36
:103AF000003800400000FF1F5118FF1F00E100E0E8
:103B0000FF00FFFF0000054070B5284C238C002B00
:103B100023D0228A002A21D1DA0023826382A38261
:103B2000E38223836383A383E38322606260A260D2
:103B3000E2601F4D1F4A6420EB8093420AD8FA22AC
:103B40000020D200934205D91B4A0A21981807F099
:103B5000BFFFC0B200232872238470BD0720E11C80
:103B6000CA7F01320240CA7705D10325201DC17FDB
:103B700001312940C17708325200A35200232100AD
:103B80001A00088A01321B180231082AF9D1221DB5
:103B9000D27F9200A350626823689B18A2689B188A
:103BA000E2689B185B099BB2C3E7C0461861FF1F20
:103BB000C061FF1FB70B000030F8FFFF30B503A84E
:103BC00004880B20002C0ED14968074D08784978ED
:103BD000090201430A20A94205D1012120001980D0
:103BE000024B1B7A137030BD192A0000C061FF1F01
:103BF000F7B5150008AA16884A680F4F147852784E
:103C0000120222430A24BA4214D10122DBB20192E9
:103C100000962A0007F0BCFC041E0BD1074B1B6862
:103C2000002B07D068782A780002104342425041A6
:103C3000013098472000FEBD022900004461FF1FAB
:103C400030B5012503790400BFB02B4211D00A49D9
:103C5000408807F009F828420BD0084B01A95B8D7A
:103C60004D800B80064B00221B7A60880B7104F09C
:103C7000DBF83FB030BDC0463C61FF1F4840FF1F2E
:103C8000C061FF1F10B50549054806F0A3FF0421D8
:103C9000044A054806F060FF10BDC0463C61FF1FA6
:103CA000FFFF0000ECBC00114840FF1F10B50248A8
:103CB00004F03CFF10BDC046413C001101230370DD
:103CC0000B4B1A7A4270022282709A78C270DA78AC
:103CD0000271032242711A7982715A79C2710C22DF
:103CE00002729A794272DB7983720B207047C04668
:103CF000C061FF1F022310B50370013B4370053301
:103D0000837010330371443B43712A33837144330E
:103D1000C37100230372064B04001B8843720A30F0
:103D2000FFF7CCFF831D0A30C0B2E37010BDC04660
:103D3000C061FF1F10B5142007F00AFF124B1422B8
:103D40000021186007F094FF002007F0A9FE012071
:103D500007F056FD022007F0FBFC032004F08AF96F
:103D6000042006F09FF9052003F0C8FB062004F0AC
:103D700095F8072001F06CFA082006F0CDFE092026
:103D800001F038F810BDC0464861FF1F07F0D0FCB5
:103D9000012007F01DFD07F073FC0000094B10B572
:103DA0000400984205D0012904D12000064906F0FC
:103DB00011FF10BD0229FCD1013904F075FE002865
:103DC000F3D0F6E7FEFF00006E61FF1F70B50D7ABD
:103DD000100004AA2C00168810221440154220D18D
:103DE000002E20D10A78022A18D14A685178157815
:103DF0000E4A09022943914205D00D4A914209D049
:103E00001C800A2404E014220A491A8007F0E0FE0C
:103E1000200070BD0C2208491A80F7E71C8001249D
:103E2000F6E70824F4E70B24F2E7C046F3FF0000AE
:103E3000F4FF0000A442FF1FD8BD001110B504001C
:103E40000749084806F0C6FE074804F0AFFD002009
:103E5000E40704D50721054A054806F07DFE10BD9C
:103E60006E61FF1FFFFF00009D3D001130BD00117E
:103E70008C40FF1F00B50C4BBFB01A780B4902A84D
:103E800000F0C0FC6B4680B2D880002809D06A469A
:103E9000074B01A91B889380064B0022188803F06A
:103EA000C3FF3FB000BDC0464C61FF1F4D61FF1F07
:103EB000E640FF1FF041FF1F00B50C4BBFB01A7862
:103EC0000B4902A801F0F6FE6B4680B2D8800028AC
:103ED00009D06A46074B01A95B8D9380064B0022EF
:103EE000188803F0A1FF3FB000BDC0467661FF1FF8
:103EF0007761FF1F8C40FF1FF041FF1FF7B50E00D9
:103F0000377A1C0008AB11003D001A8820231D40A1
:103F10001F423CD13378022B3BD173681F785B780A
:103F20001B023B431E4FBB4208D01E4FBB4214D066
:103F30001D4DAB4221D00A252800FEBD002A2AD102
:103F4000142C2AD82200F06807F042FE174B1C7090
:103F5000012CF1D9FFF7B0FFEEE7002A1BD1202C8E
:103F60001BD82200F06807F033FE114B04211C70AF
:103F7000104B187807F0BCFBDEE7E3B20124009297
:103F800001940A00310007F003FB0500D4E708257F
:103F9000D2E70125D0E70B25CEE70D25CCE7C046BB
:103FA000F3FF0000F4FF0000022900007661FF1F0C
:103FB0004C61FF1FF861FF1F332310B5040003702D
:103FC0000A220749013007F003FE064B0F201B6849
:103FD0001A0AE37222731A0C1B0E6273A37310BDCC
:103FE000C061FF1FE861FF1F30B5012503790400A0
:103FF000BFB02B4213D00B49408806F035FE284253
:104000000DD06A46084B02A81B889380FFF7D4FFA7
:104010006B46D8800022608801A903F005FF3FB0FD
:1040200030BDC0466E61FF1FE640FF1F10B502485D
:1040300004F07CFD10BDC046E93F001170B51600CC
:1040400004AA148805AA15784A68507811780002E5
:104050002A4A0843801805284BD807F0C9FB0313E8
:104060001E29343F0720042C0BD80522121BAA421C
:1040700000D92A0022491A803000091907F0A8FD4A
:10408000002070BD0720112CFBD81222121BAA425F
:1040900000D92A001B491A80EEE707200E2CF0D821
:1040A0000F22121BAA4200D92A0017491A80E3E7FF
:1040B0000720032CE5D80422121BAA4200D92A00AB
:1040C00012491A80D8E70720032CDAD80422121BE1
:1040D000AA4200D92A000E491A80CDE70720032CF6
:1040E000CFD80422121BAA4200D92A0009491A80FB
:1040F000C2E700220A201A80C3E7C046DCD5FFFFD2
:104100007BBD00119461FF1F6BBD001166BD0011E6
:1041100061BD00115CBD001110B50D21024A0348BC
:1041200006F01AFD10BDC04650BD0011FC40FF1F37
:1041300013B5104C0423217C01AA00F061F900287A
:1041400015D16B469A88236852BA92B2534322899A
:1041500009491B0C9B184B806B46DA88636852BA7E
:1041600092B2534362891B0C9B188B8016BD0120B1
:10417000FCE7C046A861FF1FC061FF1F37B5174CA1
:1041800007236A46217C00F03BF9002824D16B46C6
:104190001B787F2B20D86B46DD78F0232A041B0385
:1041A0001A406B469B880E495BBA9BB21A43236840
:1041B0002D09534322891B0C9B184B806B465A7860
:1041C0009B7812031B011A4363682A435343628995
:1041D0001B0C9B188B803EBD0120FCE7A861FF1FD4
:1041E000C061FF1F7FB50226154C0022217C03AB66
:1041F0000096050000F0D6F8002802D0012004B097
:1042000070BD0E23217C0122280000966B4400F033
:10421000C9F80028F2D16B469A892368D2BA534371
:10422000228908491B149B184B806B46DA89636806
:1042300052BA92B2534362891B0C9B188B80DEE703
:10424000A861FF1FC061FF1F70B5114C237C002BBC
:104250000FD0382B0ED10F4D280000F051F8CC2391
:10426000AC222800217C9B0100F012F9280000F00C
:1042700085F870BD084BE2899A42FAD1054D2800B5
:1042800000F03EF800222800217C00F0E3F8EDE782
:10429000A861FF1FD441FF1F8305000070B5144CB7
:1042A000237C002B1FD06369002B1CD0114D2800EC
:1042B00000F026F86369280098470400280000F001
:1042C0005DF8002C10D10C4B0422995E002905DA10
:1042D0009C801A8801321A80200070BD074A9142E2
:1042E000F7DD9A80F5E70124FEF78AFEF4E7C04681
:1042F000A861FF1FD441FF1FC061FF1F0F270000EF
:1043000070B5C17905000C00631E9C411A4BE40294
:10431000E41849000460C9B2007906F007F9E979A8
:10432000687949000131C9B206F000F9E87909302D
:10433000C0B207F05DFB0023E36661332360AA7916
:104340005B3B002A0ED022689A43023B1343236052
:104350000A23E3610733236200232363A36301334A
:10436000E36370BD22689A4302231343236046230C
:1043700063610633A361EFE70050004070B500258C
:1043800004000368DD66C0790930C0B207F090FC14
:104390002900207906F066F82900607906F062F8B5
:1043A00070BD0000F8B51E0006AB1D780023046840
:1043B0001700E366616007F05BF901238022E36682
:1043C0002B0027615200013B08D207F049FB08206F
:1043D0000A4A1168002D03D12800F8BD2261F2E7D6
:1043E000236F034203D02369013D33700136136804
:1043F0005B1A032BEED90125EEE7C0466008FF1FCC
:1044000070B51C00002305681600EB66696007F0B4
:104410002FF901238022EB6623005200013B08D2D2
:1044200007F01EFB08200A4A1168002C03D1200067
:1044300070BD2A61F2E72B6F034203D02B69013C68
:104440003370013613685B1A032BEED90124EEE7B3
:104450006008FF1F002370B504681500E366616003
:1044600007F006F90123E366256107F0F9FA8020D9
:10447000064A80001168636B034205D113685B1A1A
:10448000032BF8D9012070BD0020FCE76008FF1F56
:1044900070B51D00002304681600E366616007F034
:1044A000E7F80123E36626610F33626B1A42FCD002
:1044B0002B0A23611023626B1A42FCD0EDB22561F6
:1044C00007F0CEFA8020074A80001168636B034230
:1044D00005D113685B1A032BF8D9012070BD0020A9
:1044E000FCE7C0466008FF1F70B51E00002305688A
:1044F0001400EB66696007F0BBF80123A619EB66B0
:104500000F33B4420ED107F0ABFA80200A4A800084
:1045100011686B6B03420CD113685B1A032BF8D93B
:10452000012070BD21782961696B1942FCD00134EA
:10453000E7E70020F5E7C0466008FF1F10B5084C0C
:10454000E368002B08D18022064B52021B689B189F
:104550006360054B1B68236007F072FAA06010BD12
:10456000E861FF1FC8F00040CCF0004070B5184A69
:10457000936A916A9942FBD116498A689A421FD37D
:104580009A1A8B60144B0126186893B2D202D20E8D
:104590004343424300204C681B0A1B1912029B181C
:1045A0000E4C0A684B60551CA3420CD8002801D061
:1045B0004B600A600A4A136008680A4B186070BDB5
:1045C000581E821ADDE7084A30009B182A00EAE7E5
:1045D00000F00040E861FF1F140AFF1F40420F0077
:1045E000C8F00040CCF00040C0BDF0FF70B51F4CDB
:1045F00023793F2B01D93F2323711D4B22791A7058
:104600001878C0B207F00CF918231A491A4A0B801F
:104610001A4913800B805380A379194980200B809D
:104620000C21938001334B43164D191C000183422A
:1046300000D9011C2980D1806379002B11D101336D
:104640006371237A012B01D8022323726279237AC2
:104650000D4853430A21584307F03AFA0B4D28609E
:1046600070BDA02BEDD9A023EAE7C046DC61FF1F97
:10467000480AFF1FEE41FF1FC443FF1FEC41FF1F0D
:10468000EA41FF1FE841FF1F71020000CC61FF1FDC
:10469000F8B519210020FEF7A9FE114C011E114D9D
:1046A00009D10C22104BC1CBC1C4280007F0E0FA9D
:1046B000FFF79CFFF8BD0C2220000C49FEF76AFEB4
:1046C0000C2802D0084B43CB43C40C2228000849D5
:1046D000FEF760FE0C28EBD00C220021E5E7C04677
:1046E000DC61FF1FA861FF1FCCBD0011FC0C0000A6
:1046F000F50C0000F0B51D4C8022A5440400882074
:1047000069465201400507F03BFA902212016A44C3
:104710001300200032C832C316C816C38023144CBD
:10472000144FA6689B033343A3603B6007F0F8F97E
:104730008823A0685B05C01807F0A2F9002588232C
:1047400029008022A0685B05C01840196944520006
:1047500007F06EFA80230135FF355B019D42EED1F3
:10476000A6603E60044B9D44F0BDC046FCEFFFFFD9
:104770003443FF1F9808FF1F04100000F0B5040029
:1047800087B0002825D0684607F072F91B4C022834
:1047900006D106226946200007F0D2F8002816D07C
:1047A0006946002301250F262F00E25C0133100922
:1047B0001030874038002F00324097403A000243C3
:1047C0004A610439062BEFD16846FFF793FF07B023
:1047D000F0BD182269460A4807F0D2F96A46A300DC
:1047E000D358013305D01822FF21684607F040FA5C
:1047F000EAE70134062CF1D1E9E7C0466509FF1F5D
:1048000000090011F0B5002504000E0085B0AA4291
:1048100000D186E04B1C087801934B788978377972
:1048200009021943F3783F061B040B431F43039708
:1048300020706570252800D196E033D8112813D850
:1048400006F02EFF69002501250125012501AA009A
:10485000B800B1002501250125012501250125010B
:104860002501250105011F01232800D1DEE0DB28F9
:1048700000D02EE1042A00D8ACE01025052A05D08E
:10488000551F2A003800711D07F0A2F905223100DA
:10489000200007F09DF92A003900601D07F098F903
:1048A00005353EE0562859D010D8332800D19DE078
:1048B000552839D02628DAD19C4B2900132218001C
:1048C0001D0007F0D5F9FEF79BFB5CE0712800D1D5
:1048D00077E0722800D180E0602800D18BE0DC28EE
:1048E000C5D1022A00D875E07378BFB26370B3787F
:1048F000A370032A05D0033A390092B2F01CFEF7E8
:1049000083FC10223900E01CFEF744FDC51C002882
:1049100007DA60705CE00C222000854907F058F946
:104920000C25280005B0F0BD013A824D0C2A13D8A1
:10493000002A0AD02800019907F04AF9FFF756FE2D
:104940000C2228007C49FEF75FFC29000C22601C29
:1049500007F03EF90D25E4E70C22EBE7754D774BA8
:104960002A0043CB43C2E9E7013A704D0C2A11D823
:10497000002A08D00199280007F02AF90C22280003
:104980006F49FEF741FC29001322601C07F020F953
:104990001425C6E70C22EDE706226A49601C07F0E1
:1049A00017F90625BDE712226749601C07F010F9C8
:1049B0001325B6E708226549601C07F009F90925A7
:1049C000AFE77178F02905D8614B188801F0CEFD6A
:1049D0000225A6E7FF236370FAE75E4B012A03D0A6
:1049E00072789A706270F3E79B78F4E72000FFF723
:1049F000E3FA050095E7013A564B574D062A10D8C1
:104A0000002A10D0012128005970019907F0E0F820
:104A100001F062F829000622601C07F0D9F807258A
:104A20007FE70622EEE700225A70F3E7042A04D952
:104A30004A4D2F6007F004F8A860FFF797FD0422A5
:104A4000039003A9601C07F0C3F8052569E7444DEE
:104A5000062ADFD906222800019906F071FF0028F6
:104A6000D8D006220199280007F0B2F806223D4965
:104A70002800FEF7C9FB0123364A91780B43937057
:104A8000C8E7012AA6D07078FFF778FEA0E70128D2
:104A900000D0ECE6931E344F132B06D87378002B0E
:104AA0000BD100F015F900F04BF9304B39001D78AF
:104AB000601C6A1E07F08CF833E7551E2A00019926
:104AC000380007F085F838002949AAB2FEF79CFBA8
:104AD000E9E7DA281DD1042A00D87BE7082A15D98E
:104AE000B37972791B021343F27912041A43337AB1
:104AF0001B0613433B603B680522310020000393F3
:104B000007F066F80422601D03A956E7FE236370D0
:104B1000F1E7DE2800D05DE7511E012A01D1002512
:104B2000FFE6019800F0BEFFF9E7C046A861FF1F4D
:104B3000D8BD0011DC61FF1FFC0C0000CCBD0011D2
:104B4000F50C0000B461FF1F9461FF1F3843FF1F85
:104B5000F041FF1FD861FF1F9442FF1FE861FF1F54
:104B60006509FF1FADAC0000D963FF1FD763FF1FAE
:104B7000AEDE000070477047020010B5094B0A32E4
:104B8000094C92B2DA815A8298811882207802F018
:104B900053FB0422054B012120781A7006F0A8FD72
:104BA00010BDC046C242FF1F2264FF1F2164FF1FC9
:104BB000013870B5042809D806F01AFE0309280840
:104BC0001200234B0221187806F092FD70BD204B95
:104BD0000821187806F0CCFD00221E4B1A72F5E76A
:104BE000802200241B4B1A4D52001A8108211A689A
:104BF0002878DC7206F0B4FD2100287806F088FDE4
:104C0000012000F087FE00F067FFDFE7104B08216E
:104C1000187806F0ADFD1048FFF76CF80F4B104AFE
:104C20009B79002093800F4A13808022094B520009
:104C3000D8721A8100F06EFE00F04EFF0A4B9B788E
:104C4000002BC3D0094A136006F04AFEBEE7C046F7
:104C5000F861FF1FCC61FF1FF941FF1FDC61FF1FDF
:104C6000C443FF1FEA41FF1FD861FF1F34F000401B
:104C700010B501290BD1082809D1054B1B78002B51
:104C800005D02622034B04485A72FFF775FF10BD6A
:104C9000FA63FF1FCC61FF1FC40900000300F0B5D9
:104CA0000A4D8E18B14202D152008018F0BD0C7826
:104CB0002F6824093C5D0F271C700C7801313C40A3
:104CC0002F683C5D5C700233ECE7C046E441FF1F97
:104CD0000E22124B10B51A700D23114C114923707E
:104CE000093A043B1048637006F072FF2D2301223D
:104CF0000E490F48E371FFF7D1FF01220D49FFF77D
:104D0000CDFF01220C49FFF7C9FF030000200B492A
:104D100002001870FEF778FA10BDC046F663FF1F58
:104D2000D763FF1F7BBD0011D963FF1F6709FF1FFA
:104D3000DF63FF1F6609FF1F6509FF1FAEDE00006E
:104D400070B5134C142220001249FEF723FB431EBA
:104D5000114D132B19D8AB78002B16D0431C2B7098
:104D600009236B7000230019037028780B4B013066
:104D70002900C0B2187006F0D3FD2978220001394D
:104D8000C9B2002005F006FE70BDFFF7A1FFECE7F9
:104D9000D963FF1FAEDE0000D763FF1FF663FF1F5E
:104DA00010B5114B1A781870002A0ED000280BD1BC
:104DB0000E4B1A78062A07D85423D340DB0703D5B5
:104DC0000B4B187802F038FA10BD0028FCD0074BC6
:104DD0001B78012B02D0033B022BF5D8044B012199
:104DE000187806F085FCEFE7FA63FF1F2164FF1FC8
:104DF0002264FF1F70B5514E514A5249307008204D
:104E000005F054FC0121022005F05AFB022005F0B8
:104E10003BFC0121002005F053FB002005F034FC91
:104E200000F0E4FEFEF7ECF806F0EAFE0322464945
:104E30004648FFF733FF2D24030004221C70444929
:104E40000130FFF72BFF30230470424D424C43707A
:104E500083702E3B062220004049EB87FEF79AFA2A
:104E6000062813D0200006F003FE022809D00321F3
:104E7000200006F0B5FE8D23E3706E3B23711933DD
:104E80006371062220003549FEF7BEF9344B1B68DA
:104E9000FC335C64FFF754FF0020FFF781FF314CC7
:104EA000314A0121314B1278207802F087F9304ADB
:104EB000304B12780021207802F080F901222E4B2D
:104EC0001A702E4BDB78552B31D12D4B3B325A7259
:104ED0002C4B2D4AAB81EA812B826A8220213078CB
:104EE00006F0E6FB0120404205F0A0FD0120404213
:104EF00005F03CFEFFF710F9FEF7C4FE00F0B2FC2F
:104F000001204042FEF79AFF012006F069FCF020E4
:104F100001F010FB0121307806F0EAFB307802F056
:104F2000E7FA1A4806F01CFDFEF766FD70BD642224
:104F3000174B5B7953431A000A32CBE7F861FF1F26
:104F4000754B0011714C00113843FF1F9461FF1F16
:104F5000B461FF1FC242FF1F6509FF1FADAC000017
:104F60004464FF1F2264FF1F1842FF1FF941FF1F07
:104F7000F663FF1FD763FF1FC863FF1FD861FF1FC2
:104F8000CC61FF1FC4090000CE090000FA61FF1FB9
:104F9000DC61FF1FF8B50A0020230D001A401942FA
:104FA00063D05E4B1B78002B5CD0FFF7DFFA5C4BC5
:104FB0005C4C5D4E99686268737A8A1ADB039A4288
:104FC00002D36160FEF718FD327A217A531EDBB2FC
:104FD000994205D1FFF738F9002000F0B3FD15E044
:104FE0009142F9D300272772FFF758F9A37ABB4201
:104FF00002D0A772FEF788FD012000F0A3FD4B4F01
:105000003800FEF777FE390006F08AFB637A002B42
:1050100025D0013BDBB26372002B20D1444BDB78FF
:10502000552B01D106F05CFCE37A002B12D0002353
:10503000A27AE3729A4202D0A372FEF765FD3D4A5E
:105040003A4F1388380001331380FEF753FE3900BE
:1050500006F066FB642370795843FFF78DFD237AD1
:105060000133237220206840F8BD0BB2002B0ADA0E
:10507000314B187806F09CFD002801D006F020FD89
:1050800080200002EFE70224214206D0254B0120B8
:105090001A72FFF785FE2000E5E70B071ED5FFF724
:1050A00065FA1F4B1F49204C98684A68637A821A38
:1050B000DB039A4202D34860FEF79EFCFFF7EEF84E
:1050C000FFF7C2F8012000F03DFD00F0E5FB23688A
:1050D000DB0701D5FEF7AAFF0820C4E7CB0609D5F8
:1050E000FEF712FD0D4B1B78002B01D1FEF7DEFD04
:1050F0001020B8E70124214207D0104800F06CF8D6
:1051000006F0C6FB00F004FDC5E7042408002040BB
:105110002142A9D0FEF7AEFEBDE7C046FA63FF1FED
:10512000E861FF1FCC61FF1FDC61FF1FF941FF1F1A
:10513000D861FF1FC061FF1FF861FF1FDC41FF1F27
:10514000F0B51B4B1B4F1B883A8804001A4E1B4DB1
:1051500085B09A420DD832889A420AD3184B1A88E1
:105160002B889A4205D1174A174B12881B889A42FE
:105170001BD0052001F034FA3B8802AA1380338843
:10518000019053802B88114D93800F4B02A91B88EF
:10519000D3800F4B2A78188802F050FF0D4B08215E
:1051A0002878019A1C7006F03BFC05B0F0BDC046A3
:1051B000C663FF1FEE41FF1FEC41FF1FEA41FF1FC7
:1051C000C463FF1FC263FF1FE841FF1F2264FF1F6C
:1051D000F041FF1FC063FF1F13B50C4B1C78002C60
:1051E00011D1002801D00A4B18600A4A0A4B1178E5
:1051F0000A4A10780A4A01920A4A0092002205F0EF
:10520000C1FA200016BD1124FBE7C0462164FF1F30
:10521000BC63FF1F2064FF1F1064FF1F2264FF1F79
:10522000FC63FF1F0064FF1F10B5064B12201B78A4
:10523000052B06D1044B13221988044B187801F072
:10524000ABFB10BD2164FF1FF041FF1F2264FF1F55
:1052500010B500240122114B52421870104B1C70E3
:10526000104B1A8002F044F904220F4B21001A70EF
:105270000E480C3206F04CFC102221000C4806F0BF
:1052800047FC07220B4B1C600B4B1C700B4B1C701C
:105290000B4B1A700B4B1C7010BDC0462264FF1FD5
:1052A0002164FF1FF041FF1F2064FF1F1064FF1FD8
:1052B0000064FF1FFC63FF1FD663FF1FD563FF1F42
:1052C000F241FF1FD463FF1FF8B5174C0600257885
:1052D00006A814240078052D23D1B41F134FA5B2BE
:1052E0001824BD421DD88D1FADB2BD4219D8FA2574
:1052F0006D00AA4215D21D000D4F0A3DADB2BD4250
:105300000FD80C4C26800C4C21800C4900240A80BC
:105310000B4A1380FFF714FF0A4B0421187806F09C
:1053200027FA2000F8BDC0462164FF1F790C000059
:10533000750C0000EE41FF1FEC41FF1FEA41FF1F0B
:10534000E841FF1F2264FF1FF0B50BB20D0089B0CA
:10535000002B00DB70E1A44E307806F029FC041E1F
:1053600050D00378A22B00D122E1D02B1AD0912B60
:1053700045D143780E2B42D19C4B82889A423ED134
:105380009B4A83681278052A39D1032018567F2852
:1053900035D0984B1B68002B31D05B68002B2ED08A
:1053A00098472CE08078072829D806F021FA0428AD
:1053B000183F3F74A8D86378002B0CD101218C4B87
:1053C00019708D4B1A78002A5BD08C4B307801F025
:1053D000F5FE002855D00722854B1A7051E0617800
:1053E0000029F8D1E378002B11D0854A854B12783B
:1053F000307801F0E3FE60706378002BEBD1200081
:1054000006F05EFB80200002684009B0F0BD784BDA
:105410001B78022BF3D00121307806F071F90028B7
:10542000EAD10121307806F063F9E5E76378002BD3
:10543000D1D16F4F032807D13B78052B02D101331F
:105440003B701EE00223FBE76F4B1A886F4B029301
:10545000002A0BD01B78002B03D00121307806F0F6
:10546000DFFA3B78062B04D1013BE9E7029B1A7077
:10547000F7E7042B41D10121029B3078197006F027
:1054800037F95C4B1B68002BB9D01B68002BB6D0DA
:10549000574A107884E76378554F002B27D10622AE
:1054A000211D5B4806F094FB62895A4B5A491A80C9
:1054B000A2895A4B1A80E3890B800521397058491B
:1054C0000A80584A1380228A574B1A80574B1B7800
:1054D000012B09D11F2001F083F8FA2292004243E8
:1054E0000421307806F09CFA0022484B75E7312BF6
:1054F00000D070E70022454B1A700323A0E7062274
:105500000021434806F004FB0023454A0421138090
:10551000444A30781380444A138006F029F9082160
:10552000307806F025F9A379083B5A425341304AB6
:1055300003331370304B1B78002B06D0334B30787D
:105540001A78002A06D001F077FE0122314B524230
:105550001A8096E70121197006F0CAF8F5E70821CC
:10556000307806F005F96378002B00D047E72C4B24
:105570002D4F0293E388029A04211380294B30783F
:1055800003932389039A138063893B8006F0B8F85C
:10559000002800D033E7264B1B68002B00D12EE7F4
:1055A000039902983A88098800881B68984726E77B
:1055B0004379132B00D022E70389012B0AD11D4B1D
:1055C0001B78022B06D10821307806F0D1F8FFF7BE
:1055D0002BFE14E7052001F003F8082102003078C3
:1055E00006F01EFA0BE7C0462264FF1F05140000F8
:1055F0002164FF1FBC63FF1F1842FF1FF941FF1FFB
:10560000F663FF1FD763FF1FF863FF1FFA63FF1FD7
:10561000C963FF1FF041FF1FD063FF1FD263FF1F4D
:10562000C663FF1FC463FF1FC263FF1FC863FF1F62
:10563000B863FF1FC063FF1F8020C001014200D07C
:10564000E2E6CB0731D5324B1B78002B1DD0314E13
:1056500005AC3378052B1AD1023B23702E4B210069
:105660001B7823722D4B1B7863722D4B187801F039
:1056700049FD002809D007202A4B30701B68002BF9
:1056800003D01B68002B00D098470120BCE60E20F9
:10569000254B06221B7825492370254B1B78637008
:1056A00002ABC01806F094FAD8E7022308001840AD
:1056B000194209D0174B1B78052B03D11D4B1888B5
:1056C00006F07EFA02209FE60424214203D0FFF771
:1056D00037FD200098E6082308001840194200D141
:1056E00093E6154B1C78012C03D0022C0DD008201A
:1056F0008AE6124B124A134913481B8812880988FC
:1057000000880094FFF7E0FDF1E7FFF78DFDEEE77D
:10571000FA63FF1F2164FF1FF241FF1FD463FF1FC5
:105720002264FF1FBC63FF1FD663FF1FF341FF1FEF
:10573000D563FF1FF041FF1FC063FF1FE841FF1F3C
:10574000EA41FF1FEC41FF1FEE41FF1F10B502A809
:1057500004880B20002C10D1496808784978090288
:1057600001430C48814209D1022119800A4B598812
:105770001170DB7800205BB2537010BD074C0A201B
:10578000A142FAD102211980034B998811705B79EB
:10579000F0E7C0466E2A0000C061FF1F6F2A0000BC
:1057A000F7B5150008AA16884A680F4F1478527882
:1057B000120222430A24BA4214D10122DBB201921E
:1057C00000962A0005F0E4FE041E0BD1074B1B686F
:1057D000002B07D068782A780002104342425041DB
:1057E000013098472000FEBD022900003464FF1FED
:1057F00030B5012503790400BFB02B4225D01449F0
:10580000408805F031FA28420CD0124B01A95B8D7B
:1058100000220B8002234B800F4B5B888B806088BB
:1058200002F002FB0D49608805F01EFAC0070CD596
:105830000B4B01A91B8800220B8002234B80064BD7
:105840009B888B80608802F0EFFA3FB030BDC04685
:105850002C64FF1F1C42FF1FC061FF1F2464FF1F39
:105860007642FF1F10B5074C0749200005F0B2F93A
:105870002000064905F0AEF90721054A054805F064
:105880006BF910BDFFFF00002C64FF1F2464FF1F95
:10589000F8BD00111C42FF1F10B5024803F046F985
:1058A00010BDC046F157001170B540253F260821B4
:1058B0000B4BC207D2172A40DD789C7835408C43C9
:1058C0002A439C70DA70820701D521439970400702
:1058D00004D58022D97852420A43DA7070BDC0469E
:1058E0009442FF1F13210A4BDA788A431239014090
:1058F0000A43DA700222104202D0D9780A43DA70E1
:10590000400703D51022D9780A43DA707047C046A1
:105910009442FF1F10B5054B082419790A00A243D1
:10592000002801D022000A431A7110BD9442FF1FC3
:1059300010B5054B2024D9780A00A243002801D0D5
:1059400022000A43DA7010BD9442FF1F0821F8B507
:10595000324D334BAE7804000E40AE70984204DDF9
:1059600067232B70273B6B70F8BD2E4B984203DAF0
:10597000E0232B701A3BF6E700232B706B7083B289
:105980001A0029485F3292B2284F82422CD9002C4B
:1059900003DA5B421CB204232B70053420B20A21C7
:1059A00006F096F804B2FA239B009C4232DB0823EF
:1059B0002A7813432B706421200006F089F80A210D
:1059C00000B205F065FE09B22A787B5C13432B70A8
:1059D0000A21200006F07CF80A2100B205F058FEEA
:1059E00009B27B5C6A780AE06970002CDBDA5B4202
:1059F0001CB204232B70F5226B78092CE8DC1343CE
:105A00006B700A21200005F043FE09B27B5C1E4347
:105A1000AE70A9E7632CCEDCEDE7C0469442FF1FD1
:105A20001B4E00001DFCFFFF2A08000023BE0011D2
:105A30000823F7B5194FCD003E7904001E403E7192
:105A4000EDB2632806DD5F3333433B7140231D43D2
:105A50007D71F7BD0300093305DA20235B42334330
:105A60003B71C623F3E70E4B019300280BDA0423A6
:105A7000444224B23B710A21200005F009FE019B3B
:105A800009B25B5CE3E70928F5DD0A2106F020F89E
:105A9000019B00B21B5C1E433E71ECE79442FF1F6A
:105AA00023BE0011F8B50A4F05003B780E00002B0D
:105AB0000CD0084C2000FEF723FC33002A00200005
:105AC0003978FEF711FD2000FEF758FCF8BDC046FE
:105AD0003864FF1F9C42FF1F70B50A4E0A4D062214
:105AE0003100280005F02CFF002809D0074C3100B8
:105AF0000622280006F06CF807212000FFF7D2FFED
:105B000070BDC0469442FF1F8E42FF1F8D42FF1F93
:105B1000E622202110B50A4B1A70203A5A701C3226
:105B20009A70DA780A40DA70082219791140033A3B
:105B30000A431A71B7225A71FFF7CEFF10BDC04653
:105B40009442FF1F10B5244B5B78002B3AD10028FC
:105B500038D0224C0223E05E214B1B685B0632D515
:105B600009233221584305F0B3FF4130FF3000B222
:105B7000FFF7ECFE0520FFF797FE0422A35E194A0B
:105B80006320934205DC32331800642105F0A0FF46
:105B900000B20121FFF74CFF237A002413222000DA
:105BA0009A426041C0B2FFF7C3FE2000FFF79AFEA1
:105BB0000D4B1878053843425841C0B2FFF7AAFE92
:105BC000FFF78AFF10BD0A21053005F081FF00B202
:105BD000FFF7BCFE0320CEE7D861FF1FC061FF1FA7
:105BE000DC61FF1FDD2600002164FF1F70B500256A
:105BF0000A4C2000A571FEF783FB11233E212000F3
:105C0000074AFEF771FCA84200D13E35054B200043
:105C10001D700123A371FEF7B1FB70BD9C42FF1FF5
:105C200012BE00113864FF1F0200F0B501270A48B8
:105C30000A4E51188B1A002B00DCF0BD0824157891
:105C40004308684038404000805B013C58406D0884
:105C5000002CF5D10132EDE7FFFF000034BE00114A
:105C6000F0B500250F269D4200DBF0BD4C5D070915
:105C700044403440A400A05801357840F3E70000C8
:105C8000F0B589B06A460D000B000F2711001035E2
:105C90001C780133260024093E40167054700232ED
:105CA000AB42F5D12023024AFFF7DAFF09B0F0BD7D
:105CB00038BE0011F0B54E780B7889B036020C0072
:105CC000170001901E43012A61D9954B9E4200D8CE
:105CD00077E001339E421CD1062A17D1CA788B780F
:105CE00012021A430B791B0413434A7912061A4312
:105CF0008C4B5A6100221A705A808B4A5A608B4A28
:105D00009A608B4ADA60002009B0F0BD8822520503
:105D1000EEE7884B9E423CD182498B78002B00D025
:105D2000F6E00C2A31D10F22A3789343E2781202D5
:105D300013432279120413436279120613434B6012
:105D4000E279A07912020243207A00041043627AB9
:105D500012060243CA60E27AA07A1202024376482F
:105D60004A81834208D804236E49142201980B709B
:105D700005F02EFF1420C7E71201D21889235B0516
:105D80009A42F0D801238B70BDE7022AFAD005238E
:105D9000EAE76A4A01239642E6D1FFF745FA052F62
:105DA0000CD9E378A2781B021343227912041A4318
:105DB00063791B061343624A0393136005F090FD59
:105DC000A1E7584D2B78002B9DD1AB78002B00D14B
:105DD000A0E02B8901339BB20093B34200D091E045
:105DE000132AD4D9CF7C8B7C3F02122120001F4381
:105DF000FFF71AFF874200D08EE0002E3DD1E378F6
:105E0000A2781B0213432279E96812041A436379CA
:105E10001B06134303930A228B4212D1FF23A37064
:105E2000E370237163716B89002B09D1E37B227CC2
:105E30001B0212041343A27B13431B0901336B8122
:105E400000226B89002B8ED0002A67D16868370149
:105E50003818000B6B6900030390984205D96861FC
:105E600005F00EFEEB780133EB7068681022A11C80
:105E7000381805F0DDFE2E8145E76F89009A7B1EFC
:105E80009BB293423AD1E278A37812021A43237963
:105E900005A81B04134362796C6812061A43EB6869
:105EA00000920392211D0C22049305F091FE012023
:105EB000260004A940421036FFF7E2FE013F012F01
:105EC00017D1009A0B232861824200D04CE70422AC
:105ED0001C49200005F0ACFE042203A9686805F007
:105EE0004FFEE968039AFF23914200D13CE7F73B5C
:105EF0003AE73100FFF7C4FE1036DFE70923B74267
:105F0000A4D831E7009BB34200D9FCE607232BE776
:105F1000022329E7032327E7062325E70A2323E7AC
:105F2000FFFE0000A442FF1F00000111FFFF000060
:105F30005048593601FF0000FFFF001102FF00002A
:105F400034F00040B042FF1F10B5034C0B0001229B
:105F5000210000F06BFA10BD096100110B8870B5CB
:105F600006000D000224162B11D92B00032209492B
:105F700000F05CFA041E0AD1074B2A881B88191C02
:105F8000934200D9111C300089B200F0EFFA2000D2
:105F900070BDC046356100114A64FF1F10B54A78D4
:105FA0000400013A0B000220012A07D80A78002ACF
:105FB00004D005222000024900F038FA10BDC04686
:105FC000636100110A7810B50B0004000220002A5A
:105FD00004D007222000024900F028FA10BDC04674
:105FE0000F6200110A7810B50B0004000220002A8D
:105FF00004D009222000024900F018FA10BDC04662
:106000007562001110B5034C0B000B22210000F04B
:106010000DFA10BDA562001110B5034C0B000D2246
:10602000210000F003FA10BD1763001110B5034CF6
:106030000B000F22210000F0F9F910BD716300116F
:106040000A7810B50B0004000220002A04D01122A7
:106050002000024900F0EAF910BDC046816300113A
:10606000002310B51322190000F0E0F910BD000064
:1060700010B5034C0B001722210000F0D7F910BD1A
:10608000D3630011002310B51922190000F0CEF9D6
:1060900010BD000010B5034C0B001B22210000F0C6
:1060A000C5F910BD0D640011F7B584890D00060017
:1060B0000121002C22D000238268D3561778002BB0
:1060C0001EDA0C2C1AD90C3CA4B213194088009388
:1060D000230002F086FE431E984101307B06DB0F51
:1060E0006B703F23013C1F40A4B22870AF70AC809E
:1060F000002C07D0B3680133AB6000210800FEBD5F
:106100000020EBE7AC60F8E70B7803704B88437036
:106110004B881B0A83700B79C370042070470420DE
:10612000022B06D10020537811781B02009A0B43F2
:10613000138070470B8803700B881B0A4370022082
:1061400070470420009983420AD1537810781B02CB
:1061500003430B80D37890781B02034300204B80CD
:106160007047F8B50D004B7801240021461C0370E0
:106170002B788B4201D82000F8BD6B78B01C4F1CE7
:10618000012B10D1890069184B88022233704B888B
:10619000B9001B0A7370691805F07AFC04360434E0
:1061A000A4B2F9B2E4E7122359436B185A880431B8
:1061B00032705B8810221B0A7370691805F068FC46
:1061C00012361234ECE770B5049D14001E00052B46
:1061D00001D8042070BD637812781B0213432B8012
:1061E000E378A2781B02134302226B802A71211DDF
:1061F000681D063E05F04CFCB2B22A81E92AE8D8B7
:106200002800A11D0A3005F043FC0020E2E700232E
:1062100010B50A789A4201D8900010BD9A008A18E9
:106220005488013304705488DBB2240A4470948883
:1062300084709288120AC2700430EAE710B5110027
:10624000029C062B04D004201022142B01D010BD78
:10625000022222714B7808781B0203432380CB78FB
:1062600088781B02034363800431601D05F010FC35
:106270000020ECE710B50C788B7804315C43E4B275
:1062800003702200013005F003FC601C10BD0420E7
:10629000022B06D10020537811781B02009A0B4381
:1062A0001380704710B50C000A88023105F0F0FB2E
:1062B000208810BD70B504000D0004981100012B5A
:1062C00001D8042070BD1678527812023243028041
:1062D0000200F13255701470E125002C00D10C350C
:1062E000023B9AB24280AA42EBD80231043005F058
:1062F000CFFB0020E6E70420009983420AD15378BF
:1063000010781B0203430B80D37890781B02034361
:1063100000204B80704710B50C000A88023105F050
:10632000B7FB208810BD000070B501211E000420BD
:10633000049C0E400B4218D1CB40DDB28D4214D9E3
:106340000A49DBB2098899420FD32300EE331D704E
:106350003300580011184978165C090231430133A3
:106360002152D9B28D42F4D8002070BDBC42FF1F2B
:1063700010B50C000A88023105F08AFB208810BD98
:1063800010B50C788B7804315C43E4B203702200C2
:10639000013005F07DFB601C10BD10B511000298A6
:1063A000032B01D8042010BD14785278043B12024C
:1063B00022430280CA788C781202224342809AB229
:1063C0008280EB2AEED80431063005F061FB002014
:1063D000E9E710B50C000B8803700B881B0A4370AB
:1063E0004B8883704B881B0AC3708A88043006313F
:1063F00005F04EFBA088043080B210BD0420012BB4
:1064000003D100201378009A1370704710B50C0068
:106410000B8803700B881B0A43704A8802300431D2
:1064200005F036FB6088023080B210BDF0B589B04F
:1064300003931E4B029242000700D05A019102F0D2
:1064400020F81325061E2DD0029B01240370019B0A
:10645000002B04D0001903999847001984B26B46A9
:106460001B7A5BB2002B0FDA1021380002F01CFB04
:106470001925002813D130003219E1B202F066FC70
:10648000051E0CD10C34A4B2042304AA380005A9BB
:1064900093800696948101F0AFFD051E02D0300076
:1064A00005F0DEF9280009B0F0BDC0464864FF1FC2
:1064B00070B505000C0000280CD00020814209D0E6
:1064C00010222000044905F0E3FA01202B78237301
:1064D0006B78637370BDC04678BE0011F0B50600DE
:1064E0000D0017001C0085B002291BD000201029C8
:1064F00007D1022B07D0102B03D115E00020102C60
:1065000008D005B0F0BD69463800FFF7D1FF2A007A
:1065100069460BE069463000FFF7CAFF2200694672
:10652000380004E0022BE9D12A003900300005F0E0
:106530002FF9E6E7031CF02800D9F02303200849CF
:106540009AB2013A0B80D317034006499B189B105F
:106550000B80D30F04499B185B100B807047C0461B
:10656000C042FF1FBE42FF1FBC42FF1F034B1B88E0
:106570008B4202D3024B4000C1527047C042FF1F02
:106580004864FF1F014B4000185A70474864FF1FC2
:106590001722014B1A8070474864FF1F70B5050031
:1065A0000E2005F015FA041E13D0D023037000232B
:1065B0000622837007494570033005F069FA064BDF
:1065C0002100DA8A62811B7E2373044B187805F060
:1065D00057FB70BD6464FF1F5464FF1F1043FF1F0F
:1065E000262803D8024B4000C05A70470148FCE7F8
:1065F000C242FF1FFFFF000070B506000C00094DEE
:106600001C220021280005F083FA074B1E70074B5F
:106610001C7005F0ADF90123002801D000231220E1
:106620002B7070BD5464FF1F1043FF1F7564FF1F64
:1066300070B505000D4C0800E260A1601022002139
:10664000656005F00DFB012803D11021A06802F060
:1066500058FD10220021280005F002FB012803D17B
:106660001021606802F04DFD70BDC0465464FF1FEC
:1066700070B5041E05D1002903D006220D4805F08F
:1066800007FA0D4B1D78012D11D1002C05D10222E6
:106690001A7005F035F9280070BD00221A70074BFA
:1066A0001B78FF2BF7D02000FFF778FFF3E70025DA
:1066B000F1E7C0466464FF1F5464FF1F1043FF1FCF
:1066C000030010B5002801D1002010BD00780B4A4E
:1066D000002803D15988D1821B7913761378022BB5
:1066E000F2D10023984200D103331370044B1B787E
:1066F000FF2B01D0FFF752FF0120E6E75464FF1F94
:106700001043FF1F002911D000280CD04B7901281D
:1067100003D140225242134303E03F221340032897
:1067200002D001204B7170474022F4E70800FAE7DD
:1067300070B5094D0100287800280BD0074C0622BF
:10674000200005F0A5F921002878FFF7DBFF2000E5
:1067500005F09EFA70BDC0467464FF1F4E64FF1FB3
:1067600000290AD0012808D13F224B799343C02B3E
:1067700003D0403B5A425341981C704770B5174DA7
:1067800006002B78FF2B15D00A2005F021F9041EF6
:1067900010D0D0230370C83B8370114B11491B7874
:1067A0004670C3700622043005F072F92100287883
:1067B00005F066FA0C4B1B78012B0DD10B4B1B68B7
:1067C000002B03D09B68002B00D09847084B042176
:1067D0001878084A04F0C4FF70BDC0461043FF1F7C
:1067E0007464FF1F4E64FF1F7064FF1F9C64FF1FD3
:1067F000A064FF1F60EA0000014B98687047C04624
:106800005464FF1F014BDB68186870475464FF1F16
:10681000074B10B5DA68136801331360054B18781D
:10682000FF2803D08021C90104F062FF10BDC046DB
:106830005464FF1F1043FF1FF7B50E0002F0C8F8A5
:10684000051E1CD00E4B06621F78002F00D1077862
:10685000AB791020019305F0BBF8041E0FD0D023B4
:106860000380C73B8370019BE91DC370062204307F
:1068700005F00EF921003800E66005F001FAF7BDD9
:106880000E43FF1F014B18787047C0467464FF1F0A
:10689000054B002805D1054B1A78054B002A00D17D
:1068A000014B18007047C0466464FF1F7464FF1FEB
:1068B0004E64FF1F014B58687047C0465464FF1F69
:1068C000024B1868431E9841C0B270477864FF1F9E
:1068D000421E03000120152A03D9FF3B5A425341AF
:1068E000D8B27047F0B51C0000230E0085B00390AD
:1068F00002920B70029A934201D3002019E0E55CEA
:106900005A1CD2B2002DF8D0029851198142F4DC01
:106910000233DFB2A35C18000193FFF7D9FF002810
:1069200007D0013D019A0399EBB233708A4202D13C
:10693000E01905B0F0BDDB19DBB2DBE710B50C00E8
:1069400002F09EF803001220002B03D0210058888B
:1069500005F026F910BD000070B50E4D8400635996
:10696000002B15D0186A002801D004F061FF2B59C4
:10697000586A002801D004F05BFF2B59986A002860
:1069800001D004F055FF285904F052FF00232B5189
:1069900070BDC0468464FF1F1C4B70B504000E0020
:1069A000150099420AD11A4B1B68002B01D1122005
:1069B00070BD1B68002BFAD09847F9E7154B994238
:1069C00015D1134B1B68002B0AD01B68002B07D076
:1069D0009847002804D1104B1C70104B1D70E7E73E
:1069E00029002000FFF7AAFF0028E1D1F3E7080003
:1069F00001F0EEFF0028DAD003780320A342D7D1BC
:106A00002900300005F0CCF8D2E7C046FEFF0000B8
:106A10008064FF1FFFFF00007D64FF1F7C64FF1F79
:106A2000F7B50400808801F0D3FF0025A84203D009
:106A30000578A08802F008F81C4E3378002B1FD090
:106A4000AB421DD11A4B28001978FFF777FF0028B9
:106A500018D000233370A3790820A778A688019363
:106A600004F0B6FF011E0DD0D0230370CA3B837023
:106A7000019B477086808371280005F001F901E0D1
:106A8000002DE8D1A0880B4B8200D358002B01D0F9
:106A9000FFF762FF1721A088FFF768FDA08801F0CB
:106AA00027FDA08801F0FEFDF7BDC0467D64FF1FF5
:106AB0007C64FF1F8464FF1FF0B587B01D000CAB22
:106AC0001B88070001930DAB1B88142002930EABAB
:106AD0001B88160003930FAB1B880091049310AB27
:106AE0001B88059304F074FF041E1AD0D023037092
:106AF000CB3B47708370C670062229000430002DFE
:106B000011D004F0C5FF019B21006381029B009816
:106B1000A381039BE381049B2382059BA37405F05F
:106B2000AFF807B0F0BD04F0F3FFECE7F7B5009362
:106B300008AB1B8807000C200D001600019304F021
:106B400047FF041E13D0280001F042FF00280FD099
:106B50000078D0232370C93BA370009B21002381C0
:106B6000019B6770A580E680638105F089F8F7BD19
:106B7000014B1878EDE7C0461043FF1F13B5040022
:106B800064890389C2888188C0780094FFF7CEFFAA
:106B900013BD000010B5044C2068002803D004F099
:106BA00047FE0023236010BD8864FF1FA122F0B5BB
:106BB000818892004A43384B384F1B6804009B1869
:106BC0009D2292009B18827989B01A603B68002B45
:106BD0005FD01D78324B1B68002B04D05B68002B04
:106BE00001D000209847260008363100E079FFF7F1
:106BF000B7FD237DE0710200E0780493638A2900E9
:106C00000393238A0293E3890193A38800933300BB
:106C1000FFF752FFE378002B0BD1E289A379A1881B
:106C200002920196E27928000092012201F0DAFE38
:106C3000E0703B68002B20D0FFF7ACFF194D28789F
:106C400000281AD0184B1978FFF778FE002814D0C6
:106C50002B78E67808200793A78804F0B9FE011E78
:106C600009D0D0230370CA3B467083708780867139
:106C7000079805F005F800232B701721A088FFF76F
:106C800075FCA08801F034FCA08801F00BFD09B070
:106C9000F0BD064B9DE7C0463409FF1F8864FF1F07
:106CA0009C64FF1F7D64FF1F7C64FF1F1043FF1F58
:106CB000F8B5070008000E0001F08AFE041E18D087
:106CC0002620FFF78DFC051E00D12578062004F054
:106CD0007FFE041E0DD00021062204F019FFD023F0
:106CE0002370C23B21006770A370A680E8B204F055
:106CF000C7FFF8BDF0B585B001930AAB1B7807005C
:106D000002930BAB1B7808000D000092039301F077
:106D10005FFE061E22D0102004F05AFE041E1DD075
:106D20001022002104F0F4FE2620FFF759FC002871
:106D300000D13078D0232370C13BA370009B210089
:106D40002372019B67706372029BA580A372039BF1
:106D5000C0B2E3720C9BE36004F092FF05B0F0BD9B
:106D6000F7B50D00019001F033FE071E20D00E2074
:106D700004F02EFE041E1BD02620FFF731FC061E59
:106D800000D13E78D0232380C53B0622A370F91D95
:106D9000E01C04F07DFE019B2A0063810123DD409D
:106DA0001A401D40210022736573F0B204F068FFA1
:106DB000F7BD0000F0B585B0029010000D0017007F
:106DC0000A9E039301F004FE041E31D0029B002BA7
:106DD0002ED1039B02795B0724D51223134304228F
:106DE000002E08D10B99002905D10C99002902D158
:106DF0000D9900291AD01A430D9B2271002B00D047
:106E0000C9E0002E00D1CFE0002D00D0CCE0606AB8
:106E1000002801D004F00CFD1C21300004F0F8FE25
:106E2000606205E002239A430E33D7E79343237150
:106E3000654BBA00D458002C00D1AAE0002E10D027
:106E4000236A002B03D11C2004F082FE20625E4BDB
:106E5000BA00D358186A002803D01C22310004F06D
:106E600017FE0C9B002B12D0574CBB001D596B6AB0
:106E7000002B03D1162004F06BFE6862BB00E358C0
:106E8000586A002803D016220C9904F001FE0D9BCD
:106E9000002B11D04C4DBC006659B36A002B03D1B6
:106EA000142004F055FEB0622B59986A002803D0D4
:106EB00014220D9904F0ECFD380001F089FD051E47
:106EC00067D0414BBA00D358002B62D01A6A3420E5
:106ED000002A00D11C389A6A002A01D0143080B2EE
:106EE0000B9A002A01D01C3080B25B6A002B01D0C3
:106EF000163080B204F06CFD041E4AD01822002126
:106F000004F006FE2620FFF76BFB0190002801D15C
:106F10002B780193D0232370029B200063700A23F7
:106F2000294EA370039BBD00A371AB59A780196ABA
:106F30001830002905D01C22A06004F0A9FD200013
:106F400034307359996A002907D00300142214338E
:106F5000E060029304F09CFD02980B9B002B08D08C
:106F600003001C221C330B992061029304F090FD56
:106F700002987359596A002903D01622606104F0FF
:106F800087FD6B462100187904F07AFE3800FFF780
:106F9000E3FC05B0F0BD10220D9B0D991B69A018F4
:106FA000236204F075FD2CE70B9B002B00D13FE71B
:106FB000012D00D03CE7606A002801D004F038FCC5
:106FC0001C210B982AE7C0468464FF1F10B5044CAF
:106FD0002068002803D004F02BFC0023236010BDA0
:106FE0007864FF1F0B4B07B51A68002A01D10020F7
:106FF0000EBD6946531C012012780731FFF772FC61
:107000000028F4D002780123100018401A42EED074
:10701000EEE7C0469464FF1FF0B51F4F01203B68A8
:1070200087B0002B25D09B78059300F0B3FB002898
:1070300021D00A20FFF7D4FA04000B20FFF7D0FA82
:10704000164B05001E78731E9E413B68F6B2191D53
:10705000D878FFF757FB3B682900DA7A04330392AC
:107060009A7901930292009033002000059A04F06F
:1070700097FC07B0F0BDFFF7B5FF002805D006204C
:10708000FFF7AEFA04000720D8E70820FFF7A8FAB8
:1070900004000920D2E7C0467864FF1F7464FF1F14
:1070A00070B50A4E040033780D00FF2B0DD004207C
:1070B00004F08EFC011E08D0D0230370CE3B457037
:1070C0008370C470307804F0DBFD70BD2043FF1F77
:1070D00070B5040006200D0004F07AFC011E0AD0F1
:1070E000D0230370CD3B8370054B44701B688580B3
:1070F000187804F0C5FD002C01D0FFF767FF70BDC4
:107100007864FF1FF8B5264F06003B680D00112478
:10711000002B05D10522234B1B78134202D11224E8
:107120002000F8BD204A10241268002AF8D01278F6
:10713000002AF5D0DB0719D52B789A1E012A1AD818
:107140000C2004F005FD132438600028E8D000234B
:107150000A22437029000670023004F099FCFFF700
:107160005BFF041E0AD0FFF731FFD9E700F012FBE6
:107170000028E1D1E4E7002BE2D0D0E70B4B1B78ED
:10718000032BCDD11D20FFF72BFA094B18800028C7
:10719000C6D0084B04211878074A04F0E1FABFE78B
:1071A0007864FF1F7564FF1F9464FF1F7464FF1FE2
:1071B0007264FF1FA064FF1F60EA0000F7B501932F
:1071C000194B14001A78052306000F0012201A42EA
:1071D00021D0012920D1154B1D68002D1BD0022084
:1071E0001F2C18D8002C02D0019B002B13D0104B61
:1071F0001F221E706E1C0021300004F089FC0199D2
:107200002200300004F044FC310020002C70002FDC
:1072100006D004F0E5FBFEBD064B12201D68DCE73E
:1072200004F07EFBF7E7C0467564FF1F9464FF1F00
:107230002043FF1F9064FF1FF8B50F4E12243368E0
:10724000002B17D01B780F3C834213D100250B4F26
:107250000221387804F08CFA094B042138781D801B
:1072600004F086FA074B28001D8033685C7004F038
:1072700087FB04002000F8BD7864FF1FA064FF1F97
:107280008C64FF1F7264FF1F70B5012823D11B4C53
:107290002388002B03D01A4A1578002D07D0194BEC
:1072A0001B68002B02D01878FFF7C6FF70BD3B2B80
:1072B00002D93C3B2380F9E7134E0221307804F0D9
:1072C00057FAFA222388920002215A43307804F0B8
:1072D000A7FB2580EAE70B4B1B68002BE6D00B4B86
:1072E0001B785B07E2D5084B0221187804F040FABE
:1072F0000022024B1A80FFF769FED7E78C64FF1F5C
:107300007064FF1F7864FF1FA064FF1F7564FF1F78
:10731000F8B51E4D2868002803D004F089FA002330
:107320002B601B4E3068002803D004F081FA002344
:107330003360184F05243B7818002040234221D0A9
:10734000154800F02BFA3B78234213D0202004F09C
:10735000FFFB2860002813D02022002104F0D8FB76
:10736000202004F0F5FB041E306005D0202200210F
:1073700004F0CEFB002004E0286804F059FA2C60E9
:107380001320F8BD00F00AFAF4E7C0469464FF1F2A
:107390009064FF1F7564FF1F1443FF1F10B50A4C54
:1073A00023681A1E0ED0002808D10130587004F04E
:1073B000E7FA002805D02368002B02D00021FFF750
:1073C00087FE0122100010BD7864FF1FF7B5274E1D
:1073D000050033680191181E21D05C78244F012CE0
:1073E00030D1FFF7FFFD002825D02000FFF7F8F887
:1073F0000400412814D91F4B022118781E4A04F0BA
:10740000AFF91E4B3C3C1C80022233685A703B781B
:10741000002B14D128000199FFF75AFE0120FEBD70
:10742000FA2292004243002AEED0124B0221187831
:1074300004F0F6FAE8E7FFF7D3F80200F3E70023D9
:107440003B70EBE73B78002BE8D1032004F0C0FA57
:10745000011E08D0D0230370CC3B45708370336885
:10746000187804F00DFCFFF7B1FDD7E77864FF1F33
:107470007064FF1FA064FF1F60EA00008C64FF1FA0
:1074800010B51749838802008B4220D011D81549C6
:107490008B4217D0144900205B1899B2012907D8F4
:1074A000926811785A425341D8B2FFF7F9FD012092
:1074B00010BD0E4A00209B1807229BB29A42404101
:1074C000C0B2F5E783681878FFF768FFF0E78368D4
:1074D00099785A78090218781143FFF777FFE7E7A0
:1074E0000A20000006200000F8DFFFFFAFDFFFFFEB
:1074F000014B18707047C0462143FF1F10B5064C62
:10750000207001F041FA207804F0DAF905212078A2
:1075100000F062FD10BDC046A064FF1F0BB273B542
:107520000D00002B00DBC4E0884B187804F040FB12
:10753000041E0ED00378912B0FD0A22B00D1A1E016
:10754000834B1878FF2852D0210004F099FB0028C3
:107550004DD180200002684076BD43780F2B76D055
:1075600013D8052B70D00E2BEAD18088794B984226
:107570002BD8794B98421BD8784B9842E0D1A3681E
:107580001878591CFFF774F838E03E2BD8D183786F
:10759000032B74D06CD8012B6ED0022BD0D1704B42
:1075A0001B68002B23D05B68002B20D098471EE07F
:1075B0006C4BC0180C28C3D804F08AF81DC2C21541
:1075C0000BC20B0B0B3223C23C00674BC0180728C1
:1075D000B6D8664B1B68002B09D01B68002B06D061
:1075E000200098470AE0A3681878FFF7C7F8200042
:1075F00004F066FAADE7A068FFF762F800289FD0B4
:10760000F5E7A3681B78002BF1D0554B1B68002BC6
:10761000EDD01B68002BEAD0210055489847EDE7D4
:107620004F4B1B68002BE2D01B68002BDFD02100E2
:107630005048F3E7504B1B68002BD8D05B68002BF9
:10764000D5D021004348E9E7FFF7EAF9CFE7808882
:107650004A4B984203D04A4B984200D070E7464BC1
:107660001B68002BC3D05B68002BC0D02100D5E77E
:10767000153B012BBBD963E7FFF798FAB7E7FFF794
:107680007DFAB4E73F4B1B78042B07D100236A46F1
:1076900013800179408800F0C5FCA8E7364B1B68D1
:1076A000002BA4D05B68002BA1D00100364898477E
:1076B0009DE7012421420AD0294B1B68002B04D0EE
:1076C0005B68002B01D000209847012043E78B071F
:1076D0000AD5264B1B68002B04D05B68002B01D019
:1076E00020009847022036E70421280008400D4278
:1076F00000D131E7254E3388002B21D0013B9BB2CE
:107700003380002B1AD1FFF7DBF800280AD0204B7A
:107710001C70164B1B68002B04D05B68002B01D03B
:1077200020009847FFF7C6F8694601F001FD68465A
:10773000FEF7FEFF1D20FEF753FF308004200AE70E
:10774000024B187804F014F8F8E7C046A064FF1F55
:107750002143FF1F0E20000001200000091000003F
:107760009864FF1FFEDFFFFFAFDFFFFF9C64FF1F7A
:107770000C2000000B2000008064FF1F0D20000083
:10778000132000007564FF1FFFFF00007264FF1FDD
:107790007064FF1F10B501F09BF910BD014B18601C
:1077A0007047C0469C64FF1F0B880020162B01D831
:1077B00017230420014A13807047C0464A64FF1F04
:1077C00000207047074A03001188814207D0918842
:1077D0000020994202D1013080001018704700202B
:1077E000FAE7C046A864FF1FF0B58F7806000D00C9
:1077F000C5B01E2F15D1FFF7E5FF051E03D10024EC
:10780000200045B0F0BD00223B003100C07800925E
:1078100000F0B2FB0400A81C00F0D2FBFF23EB70C9
:10782000EEE7264B062403931B78FF2BE8D0182F96
:10783000E6D87B08224A013BDB0002929A58944624
:10784000002ADDD0029AD3185B68002BD8D00878C4
:10785000002802D14B78012B02D10624122FCFD160
:1078600007AFAB88697800976446AA68A047041EF2
:10787000C6D1AB78029A5B08013BDB00D318390014
:1078800030005B689847041E0BD1AB78042BB6D050
:10789000039A310010782200009700F06DFB04007D
:1078A000AEE76A78002AABD1AA7805A93B880871AF
:1078B00030000A704B80FEF747FBA0E72443FF1F10
:1078C00088BE00111D4B37B5050098420BD000292A
:1078D0000AD1FFF777FF002805D11948FFF772FF9B
:1078E000002800D0058037BD01291AD1FFF76AFFB3
:1078F000041EF8D001235B420380A378FF2BF2D053
:10790000FE2B07D00023E0781422009329001E33B9
:1079100000F032FBA01C00F053FB01235B426380AC
:10792000E1E70229DFD1013901F0BEF80028DAD100
:107930002800FFF747FF041EDFD1D4E7FEFF000059
:10794000FFFF0000022210B5074B52421A80074881
:1079500001325A809A80DA8000F07EFA044801F001
:1079600025F8002010BDC046A864FF1FE97700116C
:10797000C57800110388F7B50400002B02D1022559
:107980002800FEBD42680221137825485268FEF7A0
:10799000A5FD00282ED0234F01253A88002AEFD0DC
:1079A000802321885B0201259B1A9942E8DC0C2088
:1079B00004F0CEF8061E31D03B8822889C46002376
:1079C0001800019561469DB2491989B2AA421BD897
:1079D000002801D062443A8000233000082208C009
:1079E000210004F055F8104A1368002B13D100252C
:1079F0001660C5E76268022113780C485268FEF7EA
:107A00006DFD0028C7D1BAE760681D0140194181AA
:107A100001330198D6E71A001B68E6E71325AFE7A4
:107A2000F6BE00112243FF1FA464FF1FF4BE001125
:107A3000014B18707047C0462443FF1F14230A00EF
:107A400010B51A40194204D00122102101F048F863
:107A500010BD4B06F9D4012088434000F8E710B56B
:107A600014008B0604D50122102101F039F810BD55
:107A700008230A001A40194202D14BB2002B0FDA38
:107A8000102101F02DF8002808D02300F2331B78D4
:107A9000002BECD0F1342378012BE8D10020E6E76D
:107AA00003208907FAD4E2E7F0B51F00184B85B030
:107AB0001C68019002910392002C27D1200005B090
:107AC000F0BDA5683301ED186B89019A934211D37B
:107AD000029A93420ED8002F04D10A9B002B10D19A
:107AE0002C00EBE73B002978039A6868FEF7F6FC68
:107AF0000028F2D10136B6B2A388B342E1D8246897
:107B0000DAE7A3680A9A5B891380E9E70026F3E7BE
:107B1000A464FF1F37B50C000A88498801239142ED
:107B200017D3002A15D0651D23792A0002210A489F
:107B3000FEF7D4FC102300280BD02379618820881D
:107B400000242A000094FFF7AFFF0A23A04200D0D0
:107B5000230018003EBDC046F6BE001113B50A0052
:107B600008884988012388420BD8002809D00024BE
:107B7000137905320094FFF797FF0A23A04200D043
:107B80002300180016BD13B50A0008884988012390
:107B900088420BD8002809D00024137905320094BC
:107BA000FFF782FF0A23A04200D02300180016BD71
:107BB000F0B58BB003904A8808880E0001238242FA
:107BC00055D3002853D00023012704AC2370002292
:107BD000718813000092FFF767FF051E3ED02078E2
:107BE000002835D12B78022B18D167706A89830061
:107BF0000130E31880005A8069680222201803F0DF
:107C000047FF23780133DBB22370042B19D93B00E3
:107C10006889013080B2002BD9D01FE00223637045
:107C2000122358436A89231804305A806968102245
:107C3000201803F02DFF23780133DBB22370002BD3
:107C4000E5D10C4A6B899B185A425341DBB2DFE7FE
:107C50006378012BE4D12B78022BC7D022780A233A
:107C6000002A04D021000398FEF798F90023180099
:107C70000BB0F0BD0100FFFF0F4BF0B5040018681A
:107C8000002816D083685D89A54207D88288AE187F
:107C9000B44203DA12019A18934201D10068EFE767
:107CA0001E005F891036A74204D1002900D00D8044
:107CB0001800F0BD3300EFE7A464FF1F70B50500A6
:107CC0000C0008880021FFF7D7FF03000120002BDC
:107CD00004D022002800197AFFF7C1FE70BDF7B565
:107CE0000C00002501902300EE331B78AB4201D835
:107CF00000200AE06B00E65A00213000E718FFF789
:107D0000BBFF002802D126800130FEBD017A019818
:107D1000FFF794FE002802D03B882380F5E7013569
:107D2000EDB2E0E710B5040008880021FFF7A4FFDA
:107D300003000120002B03D02000197AFFF77EFEFC
:107D400010BD0000054B1B68002B01D1180004E09A
:107D50009A6852898242F6D198887047A464FF1FBE
:107D6000F0B50E27002687B0039302ABFF183E80C4
:107D700005001F4B40891400984207D02B78013032
:107D800000976A6880B2FFF78FFE060002212B7809
:107D900018486A68FEF7A2FB00280FD06C89200003
:107DA000FFF7D0FF002802D0013C0419A4B2039BC6
:107DB000002B00D01C80300007B0F0BD02212B78D2
:107DC0000D486A68FEF78AFB0028E7D102212B786C
:107DD0000A486A68FEF782FB002807D0002EDED032
:107DE0003B88A342DBD17489013CDFE76C89DEE785
:107DF000FFFF0000F6BE0011F4BE0011F2BE00113C
:107E000010B50C00FFF7DEFC03000220002B0AD0A7
:107E1000002C00D023609B781720FE2B03D0013864
:107E2000FF2B00D1002010BD73B50D0001A9040087
:107E30001600FFF7E5FF172805D0002E04D1290012
:107E40002000FEF727F976BD01221021200000F066
:107E500047FE0028F3D0F6E7014B18607047C04694
:107E6000B464FF1F37B56B469D1D0100040002225C
:107E7000280003F0ADFE2B88B02B0ED12379122BF6
:107E800009D12300FA331B78012B06D10121608828
:107E900000F0E0F801E01B2BF8D037BD10B5054B22
:107EA0000421187000F098F8FFF74CFDFEF770FB06
:107EB00010BDC046B864FF1F0020F0B50BB20F0024
:107EC00087B0834234DA274B187803F071FE051E21
:107ED0002BD00378A02B25D103AE3100FEF7E4F8B8
:107EE000041E0BD1B378DB0724D51F4B06341B6867
:107EF000002B03D03100688898470400A868002848
:107F000001D003F0ADFC002C08D1184A039B1340AC
:107F1000174A934206D0B3781B2B03D001216888FF
:107F200000F098F8280003F0CBFD80200002784094
:107F300007B0F0BD0F4B1B68002B10D031006888D4
:107F40009847041EDAD07378002BD7D1B27801A9F4
:107F50000A704B800C716888FDF7F6FFCEE70624A7
:107F6000F1E7C046B864FF1FB064FF1F00FFFF00C9
:107F700000011200B464FF1FF7B50190FC200D0052
:107F800017001E0003F024FD04001320002C12D063
:107F9000B02320002370089BF4226770658026714F
:107FA0000830002B08D0190003F072FD2100019861
:107FB00003F066FE0020FEBD089903F0A9FDF5E779
:107FC00010B5041E06D00078FD2803D803F020FC6D
:107FD000FF23237010BD00000A1F93B210B50400E8
:107FE0000220032B05D882400020024BD1529B185F
:107FF0009C7010BDD864FF1F0B8870B5043B040053
:108000000D000220032B0BD80121200000F04CFDB5
:1080100003001420002B03D02900200000F0DEFB19
:1080200070BD000007B51300034A00920A00012149
:1080300000F02CFC0EBDC0466182001107B5019214
:1080400003220092024B0A00122100F049FC0EBDEF
:10805000DF82001107B56B4601AA11800449D88060
:1080600008780633012802D1190003F079FD07BD15
:10807000B964FF1F0C4B10B518700023FF210B4A89
:108080001380138193819380094A53801370517236
:1080900093819372D174D3821375517703F028FDC5
:1080A00000F0FCF910BDC046E864FF1FD864FF1F54
:1080B000BA64FF1FF0B58DB06B46002003910C220F
:1080C0009B5E834200DBB0E05D4B187803F070FDEF
:1080D000051E00D1A4E00378902B00D09DE006AFF0
:1080E00001004688380000F013FA7968040000297E
:1080F00000D19CE03B88052B6ED13B89032B1CD91A
:1081000005AC200000F0A2F86288172A61D83989EE
:10811000131D994231D17968237804310291D9072E
:1081200038D5607800F08EF9071E06D00023037161
:108130002378012B08D0132B23D0A868002800D166
:1081400078E003F08DFB75E06288029909A800F0E1
:10815000A6F80290380000F08BF909AA2378387A43
:108160000192002231000092029A00F012F93800C8
:1081700000F064F9029B002BDFD0300000F080F9A2
:10818000DBE70378032BD8D16288029909A800F0B5
:10819000D6F8DEE7122B13D1029909A800F0B5F842
:1081A000021EEAD127498B88002BC6D0887909A9FD
:1081B0002378019161780091310000F0EAF8BCE782
:1081C000002302AA93833000617809AAFFF72AFFEF
:1081D000B3E71D4B0993F6E7042B02D09A1F012A3F
:1081E000ABD8184A043B9B00995A0029A5D0D21855
:1081F000907831003A0000F0AEF800289DD13B881D
:10820000042B03D001213000FFF724FF012C04D1FF
:10821000A868002801D003F023FB280003F050FCDD
:108220008020039B0002434018000DB0F0BD0128E0
:1082300000D182E701213000FFF70CFFEDE7C046D7
:10824000E864FF1FD864FF1F010017000B7803705C
:108250004B784370CB788A781B0213434380704776
:108260000A88030002700A88120A42700A88012AEA
:1082700006D14A8882704A88120AC2700420704768
:1082800002208242FBD14A8804309A704A88120A3E
:10829000DA708A881A718A88120A5A71EFE710B563
:1082A0000400012082420CD94B780A781B02134348
:1082B0002380834206D1CB788A781B0213436380E4
:1082C000002010BD022BFBD1CB788A781B02134310
:1082D00063804B790A791B021343A380F0E70B8874
:1082E00003700B881B0A43704B8883704B881B0AF2
:1082F000C3708B8803718B881B0A4371CB88837191
:10830000CB881B0AC3710820704703000120082A8C
:1083100014D14A780878120202431A80CA78887801
:10832000120202435A804A790879120202439A8063
:10833000CA798879120202430020DA80704710B5AA
:1083400004000120022A05D100204B780A781B0284
:108350001343238010BDF8B5060010200F00150050
:1083600003F036FB04000120002C0ED0A0230C22C9
:10837000290023806780201D002D07D003F088FB93
:108380002100300003F07CFC0020F8BD03F0C0FBAE
:10839000F6E7F7B51E00009008AB142017001D7813
:1083A000019103F015FB041E12D0A2230370019B60
:1083B00047704380099B057146710C220830002BE1
:1083C00007D0190003F064FB2100009803F058FC6B
:1083D000F7BD099903F09CFBF6E737B5041E0FD0F3
:1083E0004388002B0CD00025C1881323007A172264
:1083F00001950095FFF7CDFFFF236580637225701F
:1084000037BD000010B50C4904004A88002A09D085
:108410008B89002B05D00020CB8A0222834201D019
:1084200010BD012213000A20434300204032C854EB
:10843000C81842800472F3E7BA64FF1F0023438028
:1084400003707047094B00211A0010B55C88002C9E
:1084500006D01C79844203D10A234B43D01810BDA7
:1084600001310A330329F1D10020F8E7BA64FF1F74
:1084700010B50400407A03F0CBF9FF23637210BDFE
:108480007047043010B580B203F012FA002803D010
:108490000421494203F0ACFB10BD000070B500257B
:1084A000104CA0682580A581A580A84202D003F0C9
:1084B000D7F9A56000250C4C0C4B606D1D80230086
:1084C00058331D70A84202D003F0CAF96565002533
:1084D0006068002801D003F0C3F9013508340A2D83
:1084E000F6D170BD8065FF1F2465FF1F7465FF1FF7
:1084F00070B5041E09D1054D2880A881A880A86800
:10850000002802D003F0ACF9AC6070BD8065FF1F9D
:10851000F0B54B8885B00193002343600A790500CC
:108520000F00022A00D07BE0CA88032A17D98B6883
:108530005E7819783602DC78D8790E4399781B7A00
:1085400024021B020C43034353495BBA0B80331DC7
:1085500093421ED1042C04D0631F022B0ED901209C
:1085600015E0019A4D4B1201D35A002B06D0019809
:10857000FFF7BEFF4A4A1369013313610421B8684B
:108580002E812C80494203F033FB6860002005B047
:10859000F0BD434D042C06D0631F022B0FD9EB68AE
:1085A0000133EB60DBE7019A3C4B1201D35A002BFD
:1085B00005D00198FFF79CFF2B6901332B61374BE6
:1085C00030000293019B029A1B0101930023019941
:1085D0008C468B52130063449C8003939E81FFF76B
:1085E00050FF039B041E986016D00421B8684942CE
:1085F00003F0FEFAFA880100043A200003F048FA7A
:108600000199029AFB888A5A043B9B18029A8B5262
:108610002B6801332B60A2E7AB690133AB619EE7A6
:108620001E4B0293019B1E01029BF35A002B2DD07F
:1086300002998C19A068002828D0012A26D1FA882E
:108640009B189BB27352A189994217D39B1AC018E9
:10865000B96803F01DFA029BA289F35A934200D035
:108660007DE700222B81A3882B80A3686B60029B8F
:10867000F2520B4A53680133536070E7084A93681B
:10868000013393600198FFF733FF68E7044A5369A9
:1086900001335361F6E7C046EA64FF1F8065FF1FA0
:1086A000F064FF1F70B5051E15D10B4C0B4B1880E5
:1086B000230058331870606D002802D003F0D0F802
:1086C0006565250050356068002801D003F0C8F8C2
:1086D0000834AC42F7D170BD2465FF1F7465FF1FDD
:1086E000F0B51700A12285B0920001934243394BA7
:1086F00006001B680C009B18D933FF331D78FDF76B
:1087000041FF0430854204DD3000FDF73BFF0430BB
:10871000C5B2BD4207D33A0000213000019B03F0EF
:108720003FF805B0F0BD2900380003F031FA23000E
:10873000C6B250331E700393019B29006365380055
:1087400003F006F9CBB20293002B02D0039B013653
:108750001E7000262300503303931B78B34204D8C5
:10876000606D002831D10020DBE7029A2800002A42
:1087700004D0013B1000B34200D02800F700E719F5
:10878000387002F09DFF786000280ED03A78019989
:1087900003F07EF9019A3B780136D3180E4A019313
:1087A000D369F6B20133D361D4E7039B18706065D7
:1087B000A74205D1084A1320D36A0133D362B0E738
:1087C000606803F04DF80834F2E703F049F800233D
:1087D0006365C8E73409FF1FF064FF1FF7B50D009C
:1087E00007000421686803F003FA2B890400037072
:1087F0002B891B0A43702B8883702B881B0AC3703C
:108800002E8902250436F6B2F42E15D81B4B9F4252
:1088100014D10C2003F0DCF81135011E0CD090238C
:1088200003708E3B0371043B4380154B8460C6800C
:10883000187803F025FA00252800FEBD5C237B4351
:10884000104AD3180093583301931B78002B0FD193
:108850000300320038000099FFF742FF019B05003A
:108860001B78002BE8D13800009902F0E9FFE3E71C
:10887000054A0725536A01335362DDE7FEFF000016
:10888000E864FF1F2465FF1FF064FF1FF0B587B089
:10889000009017200F0016000193FFF7F2FD13253B
:1088A000041E19D00C98031E02D00199201D984770
:1088B000030AE370052302AAA07004309081277098
:1088C0000098667003A993800494FFF787FF051E44
:1088D00002D0200002F0C4FF280007B0F0BD000065
:1088E000F0B587B01F000CAB1B78039105930121F5
:1088F0000DAB06001C78049200F0D6F81425002871
:1089000021D02000FFF77EFD0135041E1BD0114948
:10891000059B0A7803700132D2B2131EC68001D1C2
:1089200001231A000B7022713000049B03990097F9
:10893000FFF7ACFF051E09D1230021000648074AB6
:10894000093303F0DDF8280007B0F0BD0023638091
:108950002370F8E7EC64FF1FDB8300113075000023
:10896000F8B505000E00064C064F2368002B02D018
:108970003100280098470434BC42F6D1F8BDC04607
:108980009065FF1FA465FF1F0123064A5B425380C9
:10899000002313715362044A136053609360D360E1
:1089A00013617047A465FF1F9065FF1F020000233D
:1089B00010B506499C000859002801D1625010BD2D
:1089C0000133052BF6D11320F9E7C0469065FF1F50
:1089D000034A5388181A4342584140421040704796
:1089E000A465FF1FF0B585B002930AAB1F780CABEE
:1089F0001B88009008000E0001920393FFF7E8FF28
:108A000005001120002D1BD10E48FFF7E1FF0400E7
:108A10001520002C14D006220B99A771E01D03F03D
:108A200037F8019B30002371029B29006371009B82
:108A300066802370039B6562E381FFF791FF280046
:108A400005B0F0BDFFFF000010B5FFF7C1FF040047
:108A50000220002C12D060880121FFF781FF606A9C
:108A6000002801D002F0E4FE28220021200003F0BB
:108A70004FF8012300205B426380207110BD00008D
:108A800030B5074A074C5588010013780020A542ED
:108A900004D05B1A59424B415842104030BDC04689
:108AA000A465FF1FFFFF0000084A10B501230C005A
:108AB000904208D0FFF78CFF031E04D003792340B7
:108AC0005A1E9341DBB2180010BDC046FEFF0000E5
:108AD000024B1879431E9841C0B27047A465FF1F2E
:108AE00070B504000D001600FFF772FF002804D1D6
:108AF0000D4B9C4200D0143070BD416A03790520B3
:108B0000002907D012221A40102A02D10520002E77
:108B1000F2D10F20DB06EFD5897E0C20A9428941D6
:108B2000494249420840E7E7FEFF0000030010B554
:108B3000002800D110BD0348034A41889142F9D072
:108B40009847F7E7A465FF1FFFFF0000002330B53B
:108B5000C45CCD5C6C40D4540133102BF8D130BDD3
:108B60000F23002210B5C45C64002243CA54C25CC7
:108B7000D209013BF7D210BD0200010010B520322E
:108B8000103102F0ADFF10BDF0B58BB00390102096
:108B900005931700049102F0DBFF0090102002F013
:108BA000D7FF009B13240190002B05D000280CD187
:108BB0001324009802F03CFE019B002B02D0180009
:108BC00002F036FE20000BB0F0BD102002F0C0FF16
:108BD0000600102002F0BCFF13240500002E00D177
:108BE000AEE0002819D01022002102F091FF3200DF
:108BF0002900039802F074FF041E0ED133787F2BF6
:108C000051D830000099FFF7ABFF009B1B787F2BFA
:108C100053D801990098FFF7A3FF300002F008FE37
:108C2000002D02D0280002F003FE002CC1D110203C
:108C300002F08EFF0600102002F08AFF0290002E44
:108C40007CD0002878D03A000F3223000125121181
:108C500005D00F333B4015B25A4253411BB26A1E36
:108C60001201002B33D0049BD2B298180099029ABB
:108C7000FFF76CFF013D10220021300002F048FF99
:108C8000ADB2049F2D017D19AF4242D0002C33D0EC
:108C9000300002F0CDFD029B002B00D189E71800C7
:108CA00002F0C6FD85E729003000FFF759FF2800D4
:108CB0002549009AFFF74AFFA7E729000098FFF728
:108CC0004FFF28002049019AFFF740FFA5E70F2139
:108CD0000F4004998A18D9B28F4208D9D15C06A8EE
:108CE00019540133102BF6D1029A0199C0E7791A71
:108CF00048424141C901F2E73900300006AAFFF7B6
:108D000025FF3200039806A902F0EAFE103704009E
:108D1000BAE7002CBCD13000029906AAFFF716FF73
:108D2000320006A9039802F0DBFE0822040031009D
:108D3000059802F0ADFEABE71324A9E71324AAE7D8
:108D4000002800D06EE733E7FCBE0011F0B58BB011
:108D50000F0016000225009000283FD0002A3DD0C9
:108D60000B1DDBB21800029302F0F2FE1135041E57
:108D700034D0FDF747FD05003A000099201D02F0B0
:108D800067FFEBB20393E3702B0CDBB22F0A009367
:108D90006370FFB22B0E2370A7700193FDF72CFDBB
:108DA0001022010006A802F053FF2100029A04AB32
:108DB00006A8FFF7E9FE051E0DD1039B08223370BC
:108DC000009B04A9B370019B7770F370301D02F013
:108DD0003FFFFDF71DFD200002F02AFD28000BB02B
:108DE000F0BDF0B58FB00D00149E03900492059372
:108DF000002A03D1022420000FB0F0BD002EF9D0CC
:108E00000398FFF7E5FD1424071EF4D07278337839
:108E100012021A43B3781B041343F27812061A4362
:108E2000036A0192934201D30133E3D1002D03D0B1
:108E30003B7901249B07DED50822002106A802F019
:108E400067FE059B13240433DBB21800029302F083
:108E50007FFE051ECFD0059A0499043002F0F8FE7B
:108E600004223100280002F0F3FE390010221031F4
:108E70000AA802F0EDFE2900029A06AB0AA8FFF745
:108E800083FE041E0FD1082206A908A802F0E0FE06
:108E90000822311D08A802F07BFC012807D10199A6
:108EA0000398FDF7C9FC280002F0C2FCA3E70124E7
:108EB000F9E7000070B51C4C05002368181E10D09F
:108EC000002D14D11A78002A0CD1981C083202F017
:108ED000DFFD02F035FC0135002808D123681D7044
:108EE000012070BD0A331800082202F0D1FD23686A
:108EF000002BF5D0122002F06BFD061E0DD0C12311
:108F000021680370457002311022023002F0C0FD6A
:108F100023683100587802F0B3FE206802F088FC24
:108F200000232360DCE7C046CC65FF1FF8B50400D2
:108F30002020FDF755FB0D4EA700BB590500002B67
:108F40000DD000280BD0D878FF2809D108492A0075
:108F50000C55F35907480333611802F0D1FDF8BDF1
:108F6000290002F06DFE0028F0D1F8E7E865FF1F48
:108F7000D065FF1F85A1001170B5064D84006359AF
:108F8000002B05D0D87802F043FCFF226359DA7039
:108F900070BDC046E865FF1F70B506008CB00C00C0
:108FA000150000213022684602F0B2FD3100102287
:108FB000684602F04DFE1D2021000322684402F0A5
:108FC00047FE6846FFF7D8FD2D2104000322280044
:108FD000694402F03DFE20000CB070BDF0B5070002
:108FE000160097B001931CAB1D7830221EAB009188
:108FF0000AA800211C7802F08BFD102239000AA873
:1090000002F026FE1022002102A802F081FD0722B4
:10901000310002A802F01CFE072202AB9818631E62
:109020009C41019902F014FE02AB9C732B005A1E66
:10903000934102AAD3730021102206A802F068FD12
:1090400006221D9907A802F003FE1A2002ABC018E1
:1090500006221F9902F0FCFD102200990EA802F0D2
:10906000F7FD102202AB0EA908781C78013A604087
:10907000D2B2087001330131002AF5D10AA8FFF7F6
:109080007BFD102212A904000EA802F001FD10229F
:1090900006AB0EA908781D78013A6840D2B2087074
:1090A00001330131002AF5D10AA8FFF765FD044319
:1090B00010222098E4B212A902F0CAFD200017B0D5
:1090C000F0BD70B50E0014008CB00100102268468F
:1090D0001D0002F0BDFD3100082204A802F0B8FD19
:1090E0002100082206A802F0B3FD6846FFF744FD00
:1090F00004001022280008A902F0AAFD20000CB0EC
:1091000070BDF8B506000D0000243719AC4200D33D
:10911000F8BD02F055FC030A3B70631CDBB201375B
:109120009D4203D90234F054E4B2EEE71C00EDE7AF
:1091300073B506000C000225002819D0002917D0AD
:10914000032101A8FFF7DDFF6B469A793F231A4000
:10915000013313436A463000937101A92200FFF7DF
:109160001BFF051E04D10322E01C01A902F090FCA4
:10917000280076BD03785807DA08C00FD2008000B7
:109180009B0710439B0F1843C0B2704707230B4047
:10919000C908C9000B4303707047000070B5040094
:1091A000FFF7EAFE134DA4006359002B21D0186A83
:1091B000002801D002F03CFB2B59986E002801D00A
:1091C00002F036FB2B59D86E002801D002F030FB9C
:1091D0002B59186F002801D002F02AFB2B59586F29
:1091E000002801D002F024FB285902F021FB0023C3
:1091F0002B5170BDE865FF1F0E4B8000C35870B542
:109200000C00002B0FD09D68002D0CD02B78201D5A
:109210000B706B784B70A97CFFF7B8FF2B7E237225
:109220006B69E36070BD10220021200002F070FC29
:10923000F8E7C046E865FF1F014B18607047C0465D
:10924000E465FF1F074A03008000825810B5002A1A
:1092500006D0D088984203D1012901D1FFF79EFFA3
:1092600010BDC046E865FF1FF0B5264E95B08700DB
:109270000B93BB590500099112200A92002B31D0A3
:10928000D888FFF7A5FB04001420002C2AD0280062
:1092900010A9FFF7B1FFBB591E781D6A002E23D01D
:1092A0000895FDF7EFFA07000020FDF7F1FA0790A7
:1092B000A379E61D069310AD0CA9089800F0E2FA18
:1092C0000EA9280000F0D7FA0B9B0A990493069B7D
:1092D00009980293079B0396019300970EAB0CAA83
:1092E000FFF77CFE15B0F0BDFDF7CCFA069030001C
:1092F000FDF7CEFAE31DA779079310AB060008939C
:10930000DAE7C046E865FF1F30B50C4C85002A59E6
:10931000030085B00120002A0ED018006946FFF72F
:109320006BFF2B591A78D888054B002A00D1054BC2
:109330006A46072100F0D9FB05B030BDE865FF1F84
:10934000779800118598001130B5094C850029598E
:1093500085B010226846253102F09AFB2A59112166
:10936000044BD0886A4600F0C0FB05B030BDC04653
:10937000E865FF1F2199001130B5094C8500295976
:1093800085B010226846353102F082FB2A5911213E
:10939000044BD0886A4600F0A8FB05B030BDC0463B
:1093A000E865FF1F5F990011F7B54D4F860010204B
:1093B000F4590D0002F0CCFBF3592062186A132215
:1093C00000286CD0033A29009C6802F061FBF35935
:1093D0001A780192002A58D11E6A227D317B944668
:1093E00051400122019F114201D167461740217D62
:1093F000914339432175377B4F40BC466046002777
:10940000800701D44F081740012102208F40227DA0
:1094100082433A432275377B5740BC46604600275B
:10942000400701D497080F400420227DBF008243EB
:109430003A432275627D002794466046727B424023
:109440000A4201D167460F400121627D8A433A43B7
:109450006275777B5740BC4660460027800701D481
:1094600057080F400220627D7F00824317436775D3
:10947000767B00227E40760701D4BA080A40042693
:10948000617D9200B1430A4362756A78002A08D070
:109490006278002A05D005220533DA770022100011
:1094A000FEBD04222979114205D1A17C114202D1CD
:1094B0000533033AF1E7019A21782C78002A02D18A
:1094C0000A002100140018220429E8D8042CE6D848
:1094D00005206043034A05331218525CDDE7C0469D
:1094E000E865FF1F0CBF001110B50A001121024BE7
:1094F00000F0FBFA10BDC046BB9900110B0030B55F
:1095000087B001AD2B806B4604001100981D082226
:1095100002F0BEFA2A000B212000024B00F0E5FA0F
:1095200007B030BDE399001110B50A001121024BBC
:1095300000F0DBFA10BDC046379A001113B50B00DE
:1095400011006A4613706B4604000622581C02F094
:109550009FFA6A4608212000014B00F0C6FA13BDAD
:10956000579A001110B50A001121024B00F0BDFA04
:1095700010BDC046A79A00117FB505000B4BAA008D
:10958000D4580800002C0FD0666F237FE288217822
:109590000396266F0296E66E0196A46E0094FDF780
:1095A00009FC2800FFF7FAFD7FBDC046E865FF1FF4
:1095B00010B51721FFF7E0FF10BD000070B50A00DD
:1095C0000D00064B0221040000F08FFA06002978F6
:1095D0002000FFF7D1FF300070BDC0468799001111
:1095E00070B586B000236A461370836804001D7846
:1095F000681E0A2859D801A902F0FAF8060633377E
:109600003B3F43474B4F5300180000F042F90623FD
:1096100012284BD000281BD16088FFF7D9F9082306
:10962000002813D04279002A47D1264B1A78072305
:1096300012070BD5244B1A680723002A06D0166898
:10964000002E03D0290001AAB04703006A46137018
:109650006B461B786088002B2AD1FFF767FC06B0A9
:1096600070BD180000F06CF9D4E7180000F087F91D
:10967000D0E7180000F093F9CCE7180000F0ADF93E
:10968000C8E7180000F0C3F9C4E7180000F0F6F9C5
:10969000C0E7180000F0F6F9BCE7180000F013FA74
:1096A000B8E7180000F013FAB4E707236A4613700E
:1096B00069466088FFF782FFD1E70523012AC5D1FB
:1096C000024BB8E77564FF1FE065FF1FE465FF1FED
:1096D000F8B52C4F8600F35904000D00002B40D044
:1096E000DA8882423DD15A78062A33D11A78002A84
:1096F0002ED0012099681A6A097D014206D0157B97
:10970000054203D007225A700120F8BD0220014211
:1097100004D0157B054201D00922F4E70420014260
:1097200004D0127B024201D00B22ECE7164B1B68DF
:10973000002BE9D05B68002BE6D020009847BB598E
:1097400000215B78122BDFD12000FFF715FFDBE74C
:109750000E4BECE7112A04D1002900D03225290054
:10976000F2E7002D08D12000FFF732F9002803D0DE
:10977000102302791343037121002800FDF798FAA2
:10978000C2E7C046E865FF1FE065FF1FE465FF1FF5
:1097900070B50E4E8500AB590400002B13D01B781A
:1097A000002B11D10A4B1B68002B04D05B68002BE7
:1097B00001D02000984773595B78122B03D1002108
:1097C0002000FFF7D9FE70BD024BECE7E865FF1FF4
:1097D000E465FF1FE065FF1F094B8000C3581020A0
:1097E000002B0CD01A6A002A09D09B68002B06D0E7
:1097F000127A1B7E101C9A4200D9181CC0B2704706
:10980000E865FF1F70B503000D0014000220002A58
:1098100030D000292ED013700B78081D53704B7870
:109820009370FFF7A7FCE070012002212B7A2371CF
:109830006B7B034063716A7B0A40134304226371AC
:109840006E7B1640334363716E7BF608F60033433C
:1098500063712B7B0340A371287B014000200B43E5
:10986000A371297B0A401343A3712A7BD208D2003B
:109870001343A37170BD10B50A0001000120FFF76A
:10988000C1FF10BD10B50A0001000220FFF7BAFFAA
:1098900010BD70B506000C000220002E30D000294B
:1098A0002ED07378201D0B70B3784B70F178FFF7D2
:1098B0006DFC01223579257271794B100800134037
:1098C000934010400343881010408000C9080343B0
:1098D000C9000B436373B1794B10080013409340E8
:1098E00010400343881002409200C9081343C90086
:1098F0000B4321202373FCF773FE854201D2122013
:1099000070BD2220257AFCF76BFE8542F7D82378BC
:109910001820042BF4D86378012BF1D80020EFE74E
:10992000030010B50220002909D0002B07D0032224
:10993000481C0A7019000D3202F0AAF8002010BD70
:1099400003000222080010B5002B06D0002904D025
:109950000E32591C02F09CF80022100010BD0300CA
:1099600010B50220002909D0002B07D00422481C82
:109970000A7019000C3202F08BF8002010BD10B5EF
:10998000FFF7DEFF10BD03000220002906D0002BE8
:1099900004D0052200200A701B784B70704703002A
:1099A0000220002B08D0002906D05B7800200B7025
:1099B000013B082B00D918307047030010B5022076
:1099C000002909D0002B07D00622481C0A70190074
:1099D0000A3202F05DF8002010BD10B5FFF7B0FFAD
:1099E00010BD02000B00022010B500290ED0002A85
:1099F0000CD007211970118859701188090A9970C3
:109A000011180822D81C02F043F8002010BD0300F2
:109A10000A00022010B5002B0CD000290AD099783A
:109A20005878090201431180901CD91C082202F0C9
:109A30002FF8002010BD030010B50220002909D026
:109A4000002B07D00822481C0A701900921802F057
:109A50001FF8002010BD02000B00022010B50029E5
:109A60000BD0002A09D009211970117818185970E3
:109A7000511C062202F00CF8002010BD10B5FFF7B3
:109A80005FFF10BD02000B00022010B5002A09D0B4
:109A9000002907D05178197011180622581C01F0BE
:109AA000F7FF002010BD030010B50220002909D0E7
:109AB000002B07D00A22481C0A701900063201F058
:109AC000E7FF002010BD10B5FFF73AFF10BD020000
:109AD0000B00022010B5002A06D0002904D018007F
:109AE0005178FFF753FB002010BDF0B585B017008B
:109AF0001E006A4606230500080091819380FEF748
:109B0000C0FC1324011E02900CD03800B047041E84
:109B100005D1280001A9FEF76FFA041E02D00298B1
:109B200001F09EFE2800FFF701FA200005B0F0BD0D
:109B3000F0B504008BB0019115000021102202A89D
:109B400001F0E6FF334EA700B85900283CD0C38887
:109B5000A34239D10378002B36D14278062A18D196
:109B600002000100553235310C3006ABFFF7A9FA7F
:109B7000002829D12000FFF72FFE020006A902A825
:109B800001F086FF200002A901F0DAFF01200BB0EE
:109B9000F0BD816E002917D00B8A112A28D19D4271
:109BA0000ED101981231093A01F0F2FD012807D1D6
:109BB000BB5920009D6EFFF70FFE29000200DEE773
:109BC00032212000FFF7D8FC2000FEF701FF061E1F
:109BD0001BD0416A002918D00B8AAB4215D108224C
:109BE0000198123101F0D4FD01280ED1716A0AE00A
:109BF0009D42E9D108220198123101F0C9FD0128E6
:109C0000E2D1BB59996E8A7EB9E7200001F0D0FEFF
:109C1000BCE7C046E865FF1FF0B56B4D87007E5975
:109C200085B0337802900393002B00D087E0B368AF
:109C3000346A01937078062817D101221B7D1342E4
:109C400002D0217B114218D10222134202D0217B83
:109C5000114251D10422134203D0237B134200D07E
:109C60008BE0019B5A7DEB5991E007380428F8D826
:109C700001F0BEFD032E42678300B36E002B03D1BB
:109C80001C2001F065FFB066EB599C6E002C1CD0C7
:109C900010220021200001F03BFF0298FFF79CFDFD
:109CA00001002000FFF72DFA01F08AFE208220003B
:109CB00008211230FFF725FA0298FFF78DFDA076F4
:109CC000EB592100D888FFF70FFC0822EB591CE064
:109CD000B36E002B05D01A00198AF0881232FFF7F4
:109CE0000DFC0222019B197DEB5911423DD0207BD6
:109CF00010423AD0073208E0F488FCF7DBFD01009F
:109D00002000FFF711FC0A22EB595A70029B9C00BD
:109D10002A595378073B042B11D8D088FEF758FEF8
:109D200000284ED0C3895A08D2182849029B0298AD
:109D3000CB542B5941180433254801F0E1FE05B0FE
:109D4000F0BDFCF79FFD03000120834201D10020FC
:109D50000393EB59DE88FCF79BFD0399020030006A
:109D6000FFF7ECFB019AEB59117D042211420CD054
:109D7000217B114209D00B22C7E7F688FCF73CFD96
:109D800001003000FFF7EEFB6BE7019A527D0121E5
:109D90000A4204D0607B084201D00C22B5E70221C0
:109DA0000A4204D0607B084201D00E22ADE70421B4
:109DB0000A4204D0627B0A4201D01022A5E7122297
:109DC000A3E7FA225200B0E7E865FF1FEC65FF1F2A
:109DD0008FA1001110B5064B1A780423100018400B
:109DE0001A4200D00348FFF727FA002010BDC046F2
:109DF0007564FF1F2843FF1F70B50400FFF7D4FAF6
:109E0000051E43D12000FFF77FFA234EA400A0597E
:109E10008268937CDB0708D50321036A1B790B401A
:109E2000012B02D1017F0B430377431DD97F8B1E8A
:109E3000022B0DD8022900D00121C088FCF790FF29
:109E4000042133591A7F59700A431A77280070BDCC
:109E500001290CD102231022437000210C3001F0A3
:109E600057FE305910213530FFF74BF9EEE7052941
:109E7000ECD10223D118437010220C3001F008FEFF
:109E800004233259117F0B431377EAE7082518287A
:109E9000DCD1053DDAE7C046E865FF1FF0B58BB0C1
:109EA000059143887E4F9E00F45915000493002CC1
:109EB00015D1012902D000200BB0F0BD101D57783C
:109EC0001678FFF757F9EB68320002932B7A049962
:109ED000019300903B002000FCF70CFFEBE7E388C8
:109EE000049A934201D00820E6E72378012B00D1A1
:109EF000D4E0059B581E092800D9CFE001F078FC7A
:109F000005CE0A29CC506C859AB229000498FFF737
:109F100073FFD1E7200029001022453001F0B8FD81
:109F2000B9594B78042B02D1013B4B70C3E70B00AE
:109F30000A00253335320C310498FFF795F904985F
:109F4000FFF702FA0522431E9841BB59C0005A7020
:109F5000B2E7200029001022553001F099FD049B42
:109F60004F4C9D00295904980A0006AB55320C311C
:109F7000FFF77AF929591022453106A801F008FCAB
:109F8000012808D10498FFF7F7F90590002804D1BB
:109F900006222B595A7005988EE708230593FAE795
:109FA00063780C2B7AD1E36E002B03D11C2001F0D7
:109FB000CFFDE066BB59D86E00286FD01022290073
:109FC00001F066FDBB590498DC6EFFF705FC0D221D
:109FD000A076BB595A706EE7E06E00285ED06378B9
:109FE0000D2B5BD12B8808220382A91C123001F0B3
:109FF0004FFDBB599A68517D0222114226D0186A42
:10A00000407B104222D00C32E4E763780E2B45D11E
:10A01000236F002B03D1162001F09AFD2067BB5956
:10A02000186F002803D01022290001F031FD0F2203
:10A03000BB59CFE763780F2B30D1206F0622691C04
:10A04000103001F025FDBB599A68517D0422114260
:10A0500003D0196A497B1142D5D100210498FFF73A
:10A060008BFA28E7636F002B0DD0BB59586F00287F
:10A07000F3D01022290001F00BFD0122BB595242FE
:10A080005B6F1A61E9E7142001F062FDBB5960675C
:10A090005B6F002BE9D126E72978DFE707200BE784
:10A0A000E865FF1F10B5064C207001F0F9FB062192
:10A0B0002078FDF791FF0348FEF778FC10BDC046FD
:10A0C000FB65FF1F4592001100200BB270B50D001B
:10A0D000834216DA264B187801F06AFD041E0DD073
:10A0E0000378922B0ED0A02B37D0224B1878FF2864
:10A0F0003AD0210001F0C4FD002835D180200002B3
:10A10000684070BD43780E2B0BD03E2BEDD1837889
:10A11000052B12D0082BE8D181798088FFF7D8FA77
:10A1200008E0154B82889A42DFD183681878591C61
:10A13000FEF7C0FE002817D1D7E7104B1B785B074E
:10A1400012D50F4B1B68002B0ED09B68002B0BD039
:10A15000C289811D80889847ECE7FFF741FAA06823
:10A16000002801D001F07CFB200001F0A9FCC5E72C
:10A17000FB65FF1F2143FF1F182000007564FF1FB0
:10A18000E465FF1F10B50078FFF712FA10BD10B597
:10A190000078FFF7FDFA10BD0C234343084A10B5C1
:10A1A0009B185A68002A03D0012901D1904710BD9D
:10A1B0009B68002BFBD00029F9D19847F7E7C046F0
:10A1C0001866FF1F01238340094A10B5946B1C4396
:10A1D0009463506B98435063D46B200098430129DB
:10A1E00001D120001843D063116B0B43136310BDE2
:10A1F00000800040F0B500240127154B85B0DA6BD4
:10A20000144E03921A6C0192DA64019BE3403B42C4
:10A2100017D0039DE5403D400295E5B20299280024
:10A22000FFF7BAFF316A736A002908D03900002BA2
:10A2300001D0029979402800FFF7C4FF01E0002B0C
:10A24000F9D101340C36172CDFD105B0F0BDC04672
:10A2500000800040FC65FF1F064B01215A68C24088
:10A260000A4204D01B68C3401800084070471B6DA9
:10A27000F9E7C046008000400122064B82400029D9
:10A2800003D0D9680A43DA607047D9689143D9602E
:10A29000FAE7C0460038004030B5032444430F4B72
:10A2A000E25C1B199C785D7801232D1B0135AB40C6
:10A2B000013BA340A140DB430C00122807D808490A
:10A2C00092005218116819402143116030BD054AAF
:10A2D00011680B4023431360F8E7C04653BF0011D9
:10A2E00008F0004014F00040C21F70B5D4B206233D
:10A2F000092C0BD80125084C9540002908D00021D5
:10A30000FFF7CAFF23682B4323600023180070BDAA
:10A310002368AB43F8E7C04600380040214BF0B556
:10A320001B185B78022B21D1032444431E4A1F4E85
:10A33000A35C12199478012215008540B76B013C8B
:10A34000E4B23D43A240B563194C122815D89B00D6
:10A3500000290CD117495B1899680A439A600123B8
:10A36000205C154A834011680B431360F0BD11490E
:10A370005B18996891439960F1E70E4B00290DD164
:10A3800059690A435A61225C1328E8D00123203A14
:10A3900093400A49086803430B60E7E75969914312
:10A3A0005961F0E7FC65FF1F53BF001100800040BA
:10A3B00098BF001100F00040A0F00040A4F0004061
:10A3C000F8B500241B4E1C4D1C4B1B5D012B1FD1EF
:10A3D000194A9269E2401A420BD00122B2569340C8
:10A3E0002200143AD2B2022A09D815494A69134305
:10A3F0004B61013402360C35172CE5D1F8BD002233
:10A40000B2560F499200521891680B439360F0E7DF
:10A41000022BEED1E7B23800FFF71EFF01235840B0
:10A42000C1B23800FFF77AFF3800FFF715FF6877F1
:10A43000DFE7C04625BF0011FC65FF1FFD65FF1F5C
:10A4400000F00040012202388240054B002903D071
:10A4500059690A435A617047596991435961FAE74A
:10A4600000380040F8B50E0001210F008740114A66
:10A470000400D368FD43BB43D360831E8B4201D8E5
:10A48000FFF7E0FF00212000FFF72EFF0A4A0B4BE9
:10A490005168012E05D139431B1951605E700020AF
:10A4A000F8BD2940516002221C1962709A6915405A
:10A4B0009D61F4E70038004000800040FC65FF1F0C
:10A4C000012210B58240074B002906D019680A43C3
:10A4D0001A600121FFF7C6FF10BD1968914319608A
:10A4E000F7E7C046008000400C2370B500254343C9
:10A4F0000A4A29009B181D70094B04001B185D7047
:10A50000FFF7B0FF0123A340064928000A681A4359
:10A510000A6005490A689A430A6070BD1866FF1F01
:10A52000FC65FF1F348000403080004070B504009F
:10A530000E00FF2813D003250540FFF7D5FF084A7A
:10A54000A3089B009B183F22ED00AA40AE4019686B
:10A5500020009143314319600121FFF78DFE70BD4A
:10A5600018380040F8B50C244443134B0500E41898
:10A570006368002B03D1A3681220002B1AD002229B
:10A5800001270E4B00215B195A7028002770FFF736
:10A5900069FF63681E1E08D0A3683E00002B04D02C
:10A5A0002800FFF759FE4640F6B228003100FFF7B9
:10A5B00009FE0020F8BDC0461866FF1FFC65FF1F9E
:10A5C000F7B5C420FF222B4B80001958002491437B
:10A5D0003F3A0A431A508022274F5202274E1A60F0
:10A5E000274B1D5D002D21D0A31E012B03D8012177
:10A5F000E0B2FFF727FF012D18D11F4B9B69E34005
:10A600002B4213D0E3B218000193FFF725FE01009F
:10A610000198FFF755FFE3B2143B022B1DD801212F
:10A620007156184A8D405369AB4353613B7F002BF1
:10A630000DD0E5B22800FFF795FF2800FFF70CFECC
:10A640007B7F0100834202D02800FFF7A5FD013483
:10A650000C370236172CC3D1F7BD012100237156E8
:10A66000F3568D40074A9B009B189A68AA439A604C
:10A67000DCE7C04600E100E0FC65FF1F25BF0011DC
:10A68000FD65FF1F00F0004010B501210400FFF739
:10A69000E9FE0123044A002011194B70A34091697F
:10A6A0000B43936110BDC046FC65FF1F70B50E00E3
:10A6B00015000400FFF718FF0C236343094A20002C
:10A6C0009B189D605E60FFF74DFFF021064B074A27
:10A6D0008900051E5A5002D02000FFF705FF280010
:10A6E00070BDC0461866FF1F0000FF1FF5A10011D6
:10A6F00070B5134D07202C78002C1FD19822210013
:10A700005200280001F0B4FA0123C420FF222B706C
:10A710000C4B80001C635C630B4B1C605C600B4B40
:10A72000195891433F3A0A431A50802252021A6044
:10A730000D20074A074901F09BF8200070BDC04674
:10A74000FC65FF1F00800040A0F0004000E100E039
:10A75000C1A50011C1A30011030010B50620072BED
:10A7600009D8054A137001F09BFAD7210020034B4A
:10A77000034A89005A5010BD5043FF1F0000FF1FBD
:10A780008D1BFF1F70B51D0002240C2910D8094A2B
:10A79000CA40D2070CD5FBF72FFF041E08D1059A3B
:10A7A00004992800FBF744FFFCF7B2FDFFF712FB0A
:10A7B000200070BD1210000030B50D7802232C006F
:10A7C0009C43184201D02B431C0008252300AB43B7
:10A7D000284201D02B00234320241D00A543204202
:10A7E00001D01C4325002A230D70184204D0117893
:10A7F0001E3B0B43137030BD0028FCD10C21137895
:10A800008B43F7E7F8B51D0006AB1B88140007AAB9
:10A810000E000B201778002B27D10A78022A49D185
:10A820004A68507811780002244A084380180428A6
:10A8300040D800F0DDFF03121D1B2300F06801F07B
:10A84000DFF8021CC0B2B84200D93A1CD2B22000D4
:10A85000F1682A8001F01CF906E00222F3681B88E7
:10A860002A8023701B0A63700020F8BD0622EEE7E1
:10A8700001232B80F3681B782370F5E7F368002B26
:10A8800016D008222A801A8822701A88120A62704A
:10A890005A88A2705A88120AE2709A8822719A889D
:10A8A000120A6271DA88A271DB881B0AE371DBE7A6
:10A8B0002B80D9E701202B80D7E7C04600D6FFFFC9
:10A8C000F7B516000A781D0008AB1F880C0001239D
:10A8D000022A18D14A685078117800022B4A08439E
:10A8E000801803280FD800F083FF02254439E06860
:10A8F00001F086F8C0B20723B84204D37B19019354
:10A90000152B02DD0D231800FEBDE0682A00310082
:10A91000C01901F0BDF86B4600209B88E268D05456
:10A920001B4B1B68834203D01B68834200D09847AF
:10A930000023E8E70B23002FE5D1022DE2D1737845
:10A9400032781B021343E2681380114B1B68002B03
:10A95000EED01B68002BEBD00120E8E70B23002F83
:10A96000D1D1062DCED12A003100E06801F090F857
:10A97000DEE70B23002FC6D1012DC3D1327875330A
:10A98000012AC0D8E3681A70D2E7C04600D6FFFF9C
:10A990000868FF1F70B50C001500072837D800F0B5
:10A9A00027FF041436361B36242E182015290BD801
:10A9B000184E16220021300001F0AAF822002900CA
:10A9C000300001F065F8002070BD18200229FBD18D
:10A9D0001288114B1A80F6E718200829F4D10A00D2
:10A9E0000E48290001F0F4F8EDE718200129EBD119
:10A9F0000B4B10780B49DA69FFF7DEFEE3E718200E
:10AA00000129E1D1064B10780749DA6BF4E70220FF
:10AA1000DAE7C046F067FF1FCE43FF1FC443FF1FA6
:10AA20005443FF1F7C43FF1F9C43FF1F030010B5CF
:10AA30000020DB0704D50721024A034800F08CF808
:10AA400010BDC046B0BF00115443FF1F054A0300AC
:10AA50001068002803D082889A4201D1806870472C
:10AA60000068F6E7006AFF1F0A88030008009A42A0
:10AA700004D08A8804309A4200D000207047000039
:10AA8000F8B5F22200230D4F0D4E796805004243C0
:10AA90003370994200D07B600A4C0021200001F005
:10AAA00037F800231A007C60AB4202D100203370DB
:10AAB000F8BD01332280DBB2F234F5E7F86AFF1FFC
:10AAC000F66AFF1F046AFF1F73B56B46019006000C
:10AAD000684615001980FCF74DFF041E11D1002DAA
:10AAE0000FD07689002E11D00C2001F031F800280B
:10AAF0000ED0084A0460136886808560002B02D15E
:10AB00001060200076BD1A001B68F7E70224F8E702
:10AB10001324F6E7006AFF1F012100220A4B10B53B
:10AB200049420A4C198099809A719A70084B20709A
:10AB3000012019805A60FFF7A3FF2078FCF778FF07
:10AB40000448FDF733FF10BD1068FF1F006BFF1FA7
:10AB5000F86AFF1F05AC0011022310B5002802D0CF
:10AB6000FFF7B2FF0300180010BD0000030010B58E
:10AB70000020DB0704D50421024A0348FFF7A4FFA5
:10AB800010BDC046C4BF0011D443FF1FF0B50E2650
:10AB900087B003930CAB1F8802ABF61805000800C2
:10ABA00031000292FDF768F804000120002C0FD05C
:10ABB0003088FFF74BFF03000E20002B08D05E68A3
:10ABC000002E05D021002800039B029A0097B04771
:10ABD00007B0F0BD0A4B10B5984207D101220023FF
:10ABE00052420A808B708A808B7110BDFFF73CFF48
:10ABF0000028FAD001235B42038000238370F4E72E
:10AC0000FFFF0000F8B5050001290AD1134E00240A
:10AC10003388F227AB4219D028001149FFF7DAFF39
:10AC200006E0022904D10139FDF73EFF0028EDD0EE
:10AC3000F8BD3B0063437268D018D35A002B09D08B
:10AC40003A00002100F064FF0134E4B2054B1B78A8
:10AC5000A342EED801235B423380DDE7F86AFF1F91
:10AC60001068FF1FF66AFF1F10B5FFF7FDFE030017
:10AC70000020834200D0987810BD0000F0B589B064
:10AC80001C000EAB80CB03901E8810AB1B78049287
:10AC900002930B7A0D00DB0616D42B780593022B5A
:10ACA00024D00498FFF7D2FE002812D003689C46F7
:10ACB000002B0ED0029B2200019329003B0064462A
:10ACC00003980096A04705E00498FFF7BFFE002810
:10ACD00002D10E2009B0F0BD8368002BF9D00A2202
:10ACE0002900039898470028D7D0F3E76B68587875
:10ACF0001A786B4B000210439842D2D8043B98421A
:10AD000010D2684B984242D015D8674BC018012822
:10AD1000C7D80B20002EDDD1EB681A7859683A802D
:10AD2000200028E0614BC018032800D979E000F02A
:10AD30005FFD846A789E5E4B9842B2D10B20002E54
:10AD4000C8D101233B80EB6831001B7823706889F0
:10AD5000013080B2FCF790FF3A88031E0ED00178D4
:10AD600002328A183A80428962704289120AA270BD
:10AD700059680278E01C00F08BFE06E004323A804D
:10AD800031000422601C00F0C3FE0020A2E70B206B
:10AD9000002E9FD1EB6807A91E8804233B80330A4D
:10ADA000300026706370FCF767FF051E28D004ABE7
:10ADB0009A890E2304A95B183E49C668FCF7D0FFA8
:10ADC00000280BD12B783C486A680599FBF786FB75
:10ADD000002803D1012304AA5B42D3813278022ADE
:10ADE00006D17168201D00F053FE3B8802333B8082
:10ADF0000E2304AA9B181B88A3701B0AE370C4E7E8
:10AE000004ABDE81F4E70B20002E00D062E7E96896
:10AE10000398FFF729FF02233B802070000A60702F
:10AE2000B3E70B20002E00D054E70222EB681B880A
:10AE30003A8023701B0A6370A7E7E86800F0E0FD22
:10AE4000C2B203000720B24200D243E70DD00299FC
:10AE5000DBB27118994202DB921BD3B20293029BC0
:10AE6000E9681A003B8089195AE70023F6E70B20AE
:10AE7000002E00D02EE70722EB683A801A78227065
:10AE80005A7862705A88A2705A88120AE2701A7947
:10AE90002271DA886271DB881B0AA37175E7C046EC
:10AEA000042900000228000000D8FFFFFFD6FFFFA2
:10AEB00003280000FFFF0000F4BE0011F0B58DB0C4
:10AEC0006B460020089120229B5E83423DDAA64B10
:10AED000187800F06DFE071E32D00378B02B2CD10D
:10AEE0000079023816281FD800F0DAFB17001E0080
:10AEF0001E001E0031001E0096001E001D011E00D7
:10AF000052011E0073011E00CD011E0050021E00E2
:10AF10001E001E008E021E00E302944B94491B8803
:10AF200078880B80FBF71AF83800FCF79BFF914BF1
:10AF30001B68002B01D038009847380000F0C0FD96
:10AF40008020089B0002434018000DB0F0BDEE22A7
:10AF50000021874800F0DCFD0BAA3B7B798938890A
:10AF600000923A000D32FCF79FFD0400804B1B78E5
:10AF7000002C3FD146E0804B788805937F4B410001
:10AF8000CB5A0BAE073BDBB232880293002301930E
:10AF90007B4B210006930093059BFFF76FFE744DDA
:10AFA000002810D1069B3A8A1B889A420BD13800A0
:10AFB0000599123000F0ECFB002804D02B78628950
:10AFC0009B00EB185A80162306A81B183288200015
:10AFD0007989FCF7C5FE2B7804009A00AA185188DD
:10AFE0000029C3D00133DBB22B70002807D006A99B
:10AFF000C98A9180634A12889A42BCD802E0012132
:10B0000049429180002B04D059497888FAF7DAFF39
:10B010008AE73E890A2479E000253E89574B06934A
:10B020007B88069A5B009B5A033B9D4202DB002D06
:10B03000F0D05BE0162206A812183B7B79890092BB
:10B040003A0030000D32FCF72FFD0590002858D053
:10B050004689017A7888FCF7F1FC041E44D1464BFE
:10B0600078880793069B4100C95A454B0439C9B2F9
:10B0700006AAD28A06930291019400930599079B30
:10B08000FFF7FCFD041E2FD1069B39491A88931C3B
:10B09000002D26D14B807988384B4900CB5A511965
:10B0A000033B8B4220DD059B31485B8941190B71C5
:10B0B000A91C0135C9B2EDB2059145191B0A2B71C6
:10B0C000059B2D490433181800F0E2FC2C4B059A1F
:10B0D0001B88D318DDB22C4B9E4205D00136B6B288
:10B0E0009CE749889942D6D0002D0CD0204C2800EE
:10B0F000618800F0EDFC207021007888FAF772FF7B
:10B1000012E7059CF0E7002C00D183E77B78142B35
:10B1100000D109E716493B794E800B700C71788895
:10B12000FAF712FF00E7162406ABE418210038896D
:10B13000FCF7A2FD011E00D1B7E1788822880F4CF0
:10B1400045002C5B0A4D013CE4B2029400240F4BF5
:10B1500001940095FFF792FD041E00D014E1290030
:10B160007888FAF74FFFDFE6006BFF1FC042FF1F32
:10B170001868FF1F0C68FF1F0C69FF1F4864FF1F42
:10B18000FC69FF1FBE42FF1FFFFF00001A68FF1F80
:10B19000162406ABE41821003889FCF76DFD011E6A
:10B1A00000D182E178882288AE4C45002C5BAE4D00
:10B1B000013CE4B202947C89AC4B01940095FFF70A
:10B1C0005DFD041E00D0DFE029007888FAF724FF37
:10B1D000AAE60025A44B1D803B00F6331B78A24A4B
:10B1E00078880792AB4208D99E4B1288069306993D
:10B1F00043005B5A013B9A4203DB0799FAF716FFBB
:10B2000092E616246B00FB18059306ABE418059B29
:10B2100021001889FCF730FD011E03D1059B012494
:10B220001E8973E77888924B2288069C0993430015
:10B230001B5B904E013BDBB202930023009601930F
:10B24000099BFFF71BFD041E02D0059B1E895DE7CD
:10B250007B88069A5B009B5A079A108832881218DE
:10B26000934202DC1B1A013B33807F4C0230328850
:10B270000999001900F00CFC2388328801359B18CD
:10B280002380EDB2A8E70BAA3B7B7989388900922D
:10B290003A000D32FCF708FC00250590059B002BB9
:10B2A00004D10A24002D00D16EE060E0059B78886F
:10B2B000197AFCF7C3FB0100041E63D1694C6C4B87
:10B2C000788806940993069B4400E45A694B063C2F
:10B2D000E4B20BAE32880793029401910093059972
:10B2E000099BFFF7CBFC041E4CD1079B5E491B88D2
:10B2F0001A1D002D30D14A80059B5B4C5A89631979
:10B300001A716B1C9BB2E318120A1A71162306A855
:10B3100032881B1879890598FCF722FDFF21AA1CA9
:10B320002E1D03350B00059092B2B6B2ADB20028C7
:10B3300003D006ABDB8AD9B21B0AA21865191171BA
:10B340002B714C4D301D2A884949201800F0A0FB74
:10B350002B88F618B5B2A1E74988914207D17A88BF
:10B3600006995200525AEB18053A9A42C4DC3E4CF8
:10B370002800618800F00CFC207021007888FAF722
:10B380005FFED1E5002DF2D13E89BFE6162606AB61
:10B39000F61831003889FCF76FFC3D000400FA35DF
:10B3A00000282DD0037A9B060CD400227B89398992
:10B3B000788800923A000C32FFF7E8FB041E10D0A8
:10B3C0003E8915E03088FFF741FB00281AD08368DA
:10B3D000002B17D02100122278889847041EE4D051
:10B3E000EEE72B78002B02D17888FAF739FE002699
:10B3F0002B78002B00D097E5002C00D194E585E652
:10B400000124DDE70E24DBE7162506ABED18290045
:10B410003889FCF731FC041E47D0037A9B0611D40F
:10B42000154A7B881188994203D01448814207D17C
:10B430001380134BF2261D780023D9B2A94221D3E1
:10B440000924A1E72888FFF701FB00282FD0836893
:10B45000002B2CD02100122278889847041EDFD0C0
:10B4600092E7C0464864FF1F1868FF1F1A68FF1F55
:10B470000C69FF1FFC69FF1FF86AFF1FFFFF000038
:10B48000F66AFF1F31005943546801336018615A4E
:10B490000029D2D13C0008342100F22200F0F8FA51
:10B4A00021007888FAF7E4FD3EE501246CE70E24DC
:10B4B0006AE71D4B1A887B889A4231D07888FAF760
:10B4C000E1FD31E5F223059851684343CD18C95A8F
:10B4D00000291FD03B7A012B0BD16C88AB88788870
:10B4E000AA1D0094FFF752FB041E02D000233B72FA
:10B4F0002E88F2220021280000F00AFB00232B8076
:10B50000059B0133DBB20593084B05991B78064A6E
:10B510008B42D7D801235B421380002CCED0F5E5B7
:10B52000002634000596EFE7F86AFF1FF66AFF1F52
:10B5300070B504000E001500FFF796FA031E08D13F
:10B5400031000548FFF790FA03001120002B02D0CC
:10B550001C8000209D7070BDFFFF0000F8B50B4FF0
:10B5600006003B780D001400FF2B0ED00A2000F0DF
:10B570002FFA011E09D0B1230380002346800371F6
:10B58000C5800481387800F07BFBF8BD1544FF1FAF
:10B59000F7B50F0008A90600088809A90B24098837
:10B5A000002821D10234022B1ED1557813782D02A8
:10B5B0001D432B008B4301937334002B14D1FB6884
:10B5C000300019000093FFF74FFB019C85420BD020
:10B5D0002A0030000099FFF7ABFF041E04D12A00B7
:10B5E00030007989FFF7BAFF2000FEBDF0B50E7874
:10B5F00085B003900AA805880120022E0DD14C6861
:10B600002778647824023C43054FBC4205D1039857
:10B61000DBB201960095FFF7BBFF05B0F0BDC04659
:10B6200002290000034B10B51B68002B00D098477F
:10B63000FEE7C046046BFF1F07B501A8FFF7F2FF46
:10B64000044A05480021121A00F012FBF8F7DAF854
:10B65000FEE7C046086BFF1F1844FF1F00000000F4
:10B6600001B40248844601BC604700BFD532FF1FC9
:10B6700001B40248844601BC604700BF75A90000C0
:10B6800001B40248844601BC604700BF85520100F6
:10B6900001B40248844601BC604700BF350E00007B
:10B6A00001B40248844601BC604700BF313BFF1F24
:10B6B00001B40248844601BC604700BF0124000079
:10B6C00001B40248844601BC604700BF017F00000E
:10B6D00001B40248844601BC604700BF093BFF1F1C
:10B6E00001B40248844601BC604700BF8530FF1F9B
:10B6F00001B40248844601BC604700BF0D520100FE
:10B7000001B40248844601BC604700BFC94A010039
:10B7100001B40248844601BC604700BF21240000F8
:10B7200001B40248844601BC604700BF056A0000BE
:10B7300001B40248844601BC604700BFED4A0100E5
:10B7400001B40248844601BC604700BFD91B000019
:10B7500001B40248844601BC604700BF2146010095
:10B7600001B40248844601BC604700BF5952010041
:10B7700001B40248844601BC604700BFB3520100D7
:10B7800001B40248844601BC604700BF1D3AFF1F58
:10B7900001B40248844601BC604700BFCD4C0100A3
:10B7A00001B40248844601BC604700BF0519FF1F71
:10B7B00001B40248844601BC604700BFC9A900002B
:10B7C00001B40248844601BC604700BFE538FF1F52
:10B7D00001B40248844601BC604700BFA54F010088
:10B7E00001B40248844601BC604700BF6DBC000044
:10B7F00001B40248844601BC604700BF1D3BFF1FE7
:10B8000001B40248844601BC604700BF3D180000F7
:10B8100001B40248844601BC604700BF11470100E3
:10B8200001B40248844601BC604700BFDD660100E8
:10B8300001B40248844601BC604700BF014C0100CE
:10B8400001B40248844601BC604700BF3119FF1FA4
:10B8500001B40248844601BC604700BFC56D0100C9
:10B8600001B40248844601BC604700BFD9490100C9
:10B8700001B40248844601BC604700BF0D31FF1F80
:10B8800001B40248844601BC604700BF2D2EFF1F53
:10B8900001B40248844601BC604700BFC51D0000DA
:10B8A00001B40248844601BC604700BFC9260000BD
:10B8B00001B40248844601BC604700BFE92800008B
:10B8C00001B40248844601BC604700BF5D17000018
:10B8D00001B40248844601BC604700BF6D30FF1FC1
:10B8E00001B40248844601BC604700BF993AFF1F7B
:10B8F00001B40248844601BC604700BF6571010085
:10B9000001B40248844601BC604700BF291C000006
:10B9100001B40248844601BC604700BFED3AFF1FF6
:10B9200001B40248844601BC604700BF55220000B4
:10B9300001B40248844601BC604700BFB54C010019
:10B9400001B40248844601BC604700BFF30E00000A
:10B9500001B40248844601BC604700BF090E0000E4
:10B9600001B40248844601BC604700BF3555000061
:10B9700001B40248844601BC604700BF5125000065
:10B9800001B40248844601BC604700BF691F000043
:10B9900001B40248844601BC604700BF456B01000A
:10B9A00001B40248844601BC604700BF851F000007
:10B9B00001B40248844601BC604700BF091B000077
:10B9C00001B40248844601BC604700BF2951010010
:10B9D00001B40248844601BC604700BF1D4D010010
:10B9E00001B40248844601BC604700BF4D1F0000FF
:10B9F00001B40248844601BC604700BF3139FF1FD3
:10BA000001B40248844601BC604700BFDD5201001A
:10BA100001B40248844601BC604700BFAD32FF1F3D
:10BA200001B40248844601BC604700BF8B5201004C
:10BA300001B40248844601BC604700BFADAE0000BF
:10BA400001B40248844601BC604700BF156B010089
:10BA500001B40248844601BC604700BFB139FF1FF2
:10BA600001B40248844601BC604700BF9DA90000A4
:10BA700001B40248844601BC604700BFF938FF1F8B
:10BA800001B40248844601BC604700BFF137FF1F84
:10BA900001B40248844601BC604700BFE94C010084
:10BAA00001B40248844601BC604700BFB14E0000AB
:10BAB00001B40248844601BC604700BF4936FF1FFD
:10BAC00001B40248844601BC604700BF434D0100F9
:10BAD00001B40248844601BC604700BF350E000037
:10BAE00001B40248844601BC604700BFE54800003D
:10BAF00001B40248844601BC604700BF79180000C9
:10BB000001B40248844601BC604700BFA946010059
:10BB100001B40248844601BC604700BF154D0100D6
:10BB200001B40248844601BC604700BF3D36FF1F98
:10BB300001B40248844601BC604700BFEDA5000087
:10BB400001B40248844601BC604700BF311B0000BD
:10BB500001B40248844601BC604700BF3D4B010070
:10BB600001B40248844601BC604700BFE1170000F1
:10BB700001B40248844601BC604700BFC53AFF1FBC
:10BB800001B40248844601BC604700BF6D36FF1F08
:10BB900001B40248844601BC604700BF090E0000A2
:10BBA00001B40248844601BC604700BF8D1200000A
:10BBB00001B40248844601BC604700BFF54E010055
:10BBC00001B40248844601BC604700BF252600003E
:10BBD00001B40248844601BC604700BF810E0000EA
:10BBE00001B40248844601BC604700BF055E000006
:10BBF00001B40248844601BC604700BF55490100BA
:10BC000001B40248844601BC604700BF0534FF1FF1
:10BC100001B40248844601BC604700BFF94C0100F2
:10BC200001B40248844601BC604700BF4550000093
:10BC300001B40248844601BC604700BF3D37FF1F86
:10BC400001B40248844601BC604700BF514701006F
:10BC500001B40248844601BC604700BF4551010061
:10BC600001B40248844601BC604700BF1D4B01007F
:10BC700001B40248844601BC604700BFB70E000013
:10BC800001B40248844601BC604700BF594F01001F
:10BC900001B40248844601BC604700BFC5210000D2
:10BCA00001B40248844601BC604700BF8D1BFF1FE2
:10BCB00001B40248844601BC604700BF7139FF1FD0
:10BCC0000001010302000303040305020602070248
:10BCD000080209020A030B030C020D000E030F03F6
:10BCE000100311001300140315001600BD3B0011D2
:10BCF000F13B0011000000000200000002BD001135
:10BD0000192A0F180A000000F1590000FD24000054
:10BD100041460100B5800011C9A000111D75001138
:10BD2000B97E001149530011BDAE0011954F0011AD
:10BD3000CD3D0011FD3E0011000000001616000070
:10BD4000020000004CBD0011F4FFF3FFD2FC000024
:10BD50003D400011000000000000000054757961B2
:10BD60000042312E3900303031390067697468750E
:10BD7000622E636F6D2F70767678005448303546AA
:10BD8000000000000200000098BD0011292A282AA6
:10BD9000272A262A252A242A0A180000E20400005D
:10BDA0007102000078EC0000050000007440000003
:10BDB0001027000060F0000004000000066400008E
:10BDC000204E0000000000000600000005000000FA
:10BDD0001F501D00023CB4000001190019000000B2
:10BDE000A102000030313233343536373839414220
:10BDF00043444546000000004D570011A157001173
:10BE0000000000000200000010BE00116F2A6E2A20
:10BE10001A18EAD8BC80F0FC6000000000000000A6
:10BE2000000000F505D39727B6F615F7B777E6F0CB
:10BE3000C7F27200000001A0000000006410B71DEE
:10BE4000C8206E3BAC30D9269041DC76F4516B6B48
:10BE50005861B24D3C7105502083B8ED44930FF00A
:10BE6000E8A3D6D68CB361CBB0C2649BD4D2D386C0
:10BE700078E20AA01CF2BDBDFB349B5F800000800D
:10BE800000100000000000001F610011A9770011E0
:10BE900043610011B17B0011C7610011877B001164
:10BEA0003D6200115D7B00118F620011257D001144
:10BEB000F7620011257D001129630011DF7C00115C
:10BEC0003D620011157B0011B5620011BD7C0011AF
:10BED00000000000000000009B630011BD7C001109
:10BEE000FD630011C1770011052A042A012A002AE6
:10BEF000022903280128002801180018000000006A
:10BF000000000000000000000000008701010201A5
:10BF10000201010201020303040103010101010105
:10BF20000303020103000D000E00100011001300B6
:10BF30001401070108010A010B011C011D02040282
:10BF400005020702080219021A021C021D0301035E
:10BF5000020317000201000504000807000B0A0095
:10BF60001716001D1C010201010504010E0D01112F
:10BF700010011413011716011A19020201020B0A0B
:10BF8000020E0D021110021413021716030504030A
:10BF90000807030B0A030E0D0001020307090A0B31
:10BFA0000E0F101112141718191A1B1F202122002E
:10BFB00005A80011C1A80011000000000200000047
:10BFC000FABE001100000000EDB5001100000000F5
:08BFD00002000000F8BE0011A0
:020000041FFFDC
:1000000000000000353D001108BD001104BD0011C5
:100010004861FF1F00000000000000000000000019
:1000200000000000000000000000000000000000D0
:1000300000000000000000000000000000000000C0
:1000400000000000000000000000000000000000B0
:1000500000000000000000000000000000000000A0
:100060000000000000000000000000000000000090
:100070000000000000000000000000000000000080
:100080000000000000000000000000000000000070
:100090000000000000000000000000000000000060
:1000A0000000000000000000000000000000000050
:1000B0000000000000000000000000000000000040
:1000C0000000000000000000000000000000000030
:1000D0000000000000000000000000000000000020
:1000E0000000000000000000000000000000000010
:1000F0000000000000000000000000000000000000
:1001000000000000000000000000000000000000EF
:1001100000000000000000000000000000000000DF
:1001200000000000000000000000000000000000CF
:1001300000000000000000000000000000000000BF
:1001400000000000000000000000000000000000AF
:10015000000000000000000000000000000000009F
:10016000000000000000000000000000000000008F
:10017000000000000000000000000000000000007F
:10018000000000000000000000000000000000006F
:10019000F932FF1F5931FF1FC16601000000000046
:1001A000000000000000000000000000000000004F
:1001B000000000000000000000000000000000003F
:1001C000000000000000000000000000000000002F
:1001D000000000000000000000000000000000001F
:1001E000000000000000000000000000000000000F
:1001F00000000000000000000000000000000000FF
:1002000000000000000000000000000000000000EE
:1002100000000000000000000000000000000000DE
:1002200000000000000000000000000000000000CE
:1002300000000000000000000000000000000000BE
:1002400000000000000000000000000000000000AE
:10025000000000000000000000000000000000009E
:10026000000000000000000000000000000000008E
:10027000000000000000000000000000000000007E
:10028000000000000000000000000000000000006E
:10029000000000000000000000000000000000005E
:1002A000000000000000000000000000000000004E
:1002B000000000000000000000000000000000003E
:1002C000000000000000000000000000000000002E
:1002D000000000000000000000000000000000001E
:1002E000000000000000000000000000000000000E
:1002F00000000000000000000000000000000000FE
:1003000000000000000000000000000000000000ED
:1003100000000000000000000000000000000000DD
:1003200000000000000000000000000000000000CD
:1003300000000000000000000000000000000000BD
:1003400000000000000000000000000000000000AD
:10035000000000000000000000000000000000009D
:10036000000000000000000000000000000000008D
:1003700039B600110000000000000000000000007D
:10038000000000000000000000000000000000006D
:10039000000000000000000000000000000000005D
:1003A0000000000000000000000000000D1BFF1F07
:1003B000000000000000000000000000000000003D
:1003C000000000000000000000000000000000002D
:1003D000000000000000000000000000000000001D
:1003E000000000000000000000000000000000000D
:1003F00000000000000000000000000000000000FD
:08183800106FFF1F4118FF1F94
:10184000024981F3088802F0C7FA0000106FFF1FF9
:1018500070B500241E491F4A1F484C6308CA1B0567
:101860001B0DE4188242F9D11C4B80228B630021AE
:1018700009201B4B920519621A4B1B4DDA671B4B53
:10188000DA688243DA609A68194802409A60112047
:10189000296002F08DF8112002F06AF880226B6C4A
:1018A000112093436B64EE23DB006343114A1B0C4E
:1018B00013840122104B9A7201F004FC0F4B1B7829
:1018C000002B04D10E4B1021187802F095FB70BD4F
:1018D000000005408805054000060540FF010000A6
:1018E00000F0004004E100E0003800403CF000401F
:1018F000FFDFFFFF1861FF1FCC61FF1FFA63FF1FAF
:10190000F861FF1F10B502F0DFFA072804D0122893
:1019100008D0022808D010BD044A0420136B0133FC
:101920001363F8E70220F6E71420F4E7F064FF1FE2
:10193000F8B507000C0026002500503630785135E8
:10194000002804D10300287058342370F8BD29788A
:10195000CA00481E8141A3183800A25C5B68C9B266
:10196000FFF7D0FF00280DD12B78DA00A218013341
:1019700050602B703378044A013B3370136A013393
:101980001362D8E70123DFE7F064FF1F5C234343C2
:10199000074910B5C9180B0058331B78012B05D126
:1019A000FFF7C6FF034A936A0133936210BDC04636
:1019B0002465FF1FF064FF1F10B502F02DF9064AE1
:1019C0000121130010CB4942D967044B136002F088
:1019D00083FA200010BDC04600E100E010001000B6
:1019E00010B5040002F018F9024B1C6002F074FA02
:1019F00010BDC04600E100E0431E5A425341A02200
:101A0000F0B5D2015B421340154D164A40019B18B8
:101A10002A18127E8BB00191002A1BD01A000832BE
:101A2000D46F0022E6B206AFE4B294420EDC28186E
:101A3000C369002B08D0019902AA117106AA049269
:101A400002AA167303A898470BB0F0BD1978B954D1
:101A50000132EAE71A7D1A7806AB01261A70E6E72A
:101A6000B067FF1F00400040F0B5254B0400400167
:101A7000C25C85B0002A2BD01A18117E002927D00D
:101A8000917E002924D01179022921D11689D78885
:101A9000D168F51BADB22A1C102D00D9102292B2CC
:101AA000BE4217D11818012303710023C269C380F5
:101AB00003819A4206D068460321037301710293A1
:101AC00001A890470820002C00D0192001F0FAFA54
:101AD00005B0F0BD013C65426C41A0256442ED01BA
:101AE0002C40084D1B186419074D0633013A92B279
:101AF000AA42EDD01888461C1E80085C2070F5E7CD
:101B0000B067FF1F00400040FFFF00000F220E4B98
:101B100010B59868104002380A280BD801F0FEFF73
:101B20000D0A0B0A0A110A0A0A0A060002210020FD
:101B3000FFF762FF10BD0121F9E70020FFF794FFD6
:101B4000F8E7DB6FF6E7C046004000400F220E4B7F
:101B500010B59868104002380A280BD801F0DEFF53
:101B60000E0A0B0A0A120A0A0A0A060002210120BA
:101B7000FFF742FF10BD01210800F9E70120FFF740
:101B800073FFF7E7DB6FF5E70090004013B5334CC8
:101B90002378072B3DD8324B1A78324B002A39D1A3
:101BA0008022196852020A431A60252001F0C0FE03
:101BB00020232D4A11680B43802113606B460422B9
:101BC000C90508680733104228D080210422C905BE
:101BD000C86810422ED080212020C905CA688243DF
:101BE000CA6014221A701A78002A2FD18021C905E0
:101BF000C86820320243CA6014221A701A78002A78
:101C000028D11A4B1A7D22785A601D221A70593237
:101C1000DA6013BD1A6816490A40C5E7086802432E
:101C20000A6014221A701A78002ACED01A78013A63
:101C3000D2B2F7E7C8680243CA6014221A70197852
:101C40004A1ED2B21A700029F9D1C4E71A78013AB3
:101C5000D2B2C7E71A78013AD2B2CEE75043FF1F9B
:101C60001844FF1F3CF000404843FF1F0020004085
:101C7000FFFFFEFF564B70B51B68012B03D1554A81
:101C8000936D0133936502F05FF9534B534A18602B
:101C9000534B544C1A600123534A1360534A136048
:101CA0002378002B06D006225149524801F06CFFE0
:101CB00000232370504A514B10681B78C1B2002B8F
:101CC0000ED14F4CC0B223785BB2002B4FDB237890
:101CD00024785BB264B21B0424021B191B18136026
:101CE0000B1C50294ED95023464A47491078DBB285
:101CF000FF2202284BD10868444C454D267890437A
:101D00002A78964254D9227824782E78023B5D10A6
:101D1000A31B6B435201D31A10335B1118430860A5
:101D200001F02AFF031F012B45D83A4B1B78002BEB
:101D300006D0394B1B78002B02D0002002F034F97A
:101D4000A122364B92009978354B4A431B689B1869
:101D5000832292009B181B78033B012B03D8AF20F2
:101D6000400001F081FF01222E4BDA8270BD237802
:101D700024785BB264B2FF33FF341B0424021B19C6
:101D80000138ABE7CAB2022AAED20223ACE7086838
:101D9000254C264D267890432A78964208D92278F9
:101DA00024782D78023B5B10641B63435201B2E739
:101DB0002378DBB2B2E70228D5D11D4B1B78013B5B
:101DC000022B03D91B4B1B78022BCCD16C20C8E70C
:101DD0009809FF1FFC0FFF1F3C64FF1FFF3F00001F
:101DE000141003404064FF1F0C1003400010034018
:101DF000D50BFF1F7211FF1FB40003408C09FF1F9A
:101E0000680AFF1F490AFF1F94000340460AFF1F8C
:101E1000470AFF1FF908FF1F2209FF1F300DFF1F90
:101E20003409FF1FBC0BFF1F440AFF1F450AFF1F99
:101E30001C09FF1F2309FF1F10B501F0D5FF002269
:101E4000014B1A8010BDC0463A64FF1F10B501F067
:101E5000EBFFA121054A89009478054A6143126885
:101E6000044B5218528C1A8010BDC046300DFF1F13
:101E70003409FF1F3A64FF1F10B50D4B0D4A9978C6
:101E8000A1239B004B431268D218531DD97F0A4BE4
:101E90001B88994209D2441C07D0C82805D0D269B2
:101EA0005B1A5A43054B5343C01801F085FF10BD20
:101EB000300DFF1F3409FF1F3A64FF1F710200003D
:101EC00070B5244D2B68002B28D001F025FF2B681E
:101ED000D8402B680400002B27D002F07DF82B6837
:101EE000D8401D4B1D4A9978A1239B004B43126893
:101EF000D118D25C91239B00002A20D0CA5801320D
:101F0000CA50174B17491B680868834214D3D23B49
:101F1000181A012A1AD0144B186070BD01F0FCFE8B
:101F2000124B196801F070FFD3E702F055F80F4B20
:101F3000196801F069FFD4E70D495B18E8E7CA505A
:101F40000C4B1B68DB68E418201AE4E7F530FF301F
:101F5000E1E7C0461C08FF1F300DFF1F3409FF1FBB
:101F60009C09FF1F3C64FF1FA009FF1F1808FF1FEB
:101F70002DFF3F004464FF1F70B504000D002829A9
:101F800016D10300A433C2881B889B1A0B4A9BB24C
:101F900093420DD906006A3605223100653001F002
:101FA000F3FF002804D13100200002F00DF870BDCD
:101FB0002900200001F0E8FEF9E7C046FE7F00009E
:101FC000F8B50500012001F0D7FF134CA36AA26AFF
:101FD0009342FBD1114E336001F08EFE1049030095
:101FE00008601048426894460F4A17680022BC45B2
:101FF00001D24268BA1A0D4802603268AD18A422B4
:10200000E562606A520302436262094A1278002A5A
:1020100001D00F3B0B60F8BD00F00040340AFF1FF9
:10202000E408FF1F28100040180AFF1F1C0AFF1FAA
:102030001C09FF1F70B580241025E405A3682B43FD
:10204000A36001F011FFA368AB43A36070BD000063
:10205000F7B5160080221C001023D205019191686B
:1020600005000B43936000225A4BD7301A6001F0F1
:10207000D3FE9D232A002F009B00EB58CA3201217A
:102080000092FC37002B01D00021009A386801F043
:1020900093FD2900009BCB311A784F4BD3351A6042
:1020A0004B780A781B0213438A7812041A43CB78C0
:1020B0001B061343494A1BBA13604B790A791B026A
:1020C00013438A7912041A43CB7931001B06134358
:1020D000434A1BBA13606B782A781B021343AA7811
:1020E00012041A43EB781B0613433E4A1BBA1360D3
:1020F000019A330213433C4A13603C4B22001B1BE2
:102100009C4603293DDCB3089A0013005142B21AE1
:10211000032A46D1354AE018511A827840781204D1
:1021200000020243E05C043302430A600022FF2BFA
:102130004BDDF0222E4B12011A600F222D4B1A603C
:102140002D4A1368002BFCD00023224A2749136034
:10215000091B321D0B191B68043A180A23706070A2
:10216000180C1B0EA070E3700434002AF2DC8022ED
:1021700010213B68D20501333B6093688B43936029
:10218000F7BD6346D578981893782D061B042B432A
:10219000157804392B43557804322D022B43036004
:1021A000AFE7022A0AD1114AE05C511AE2185278CC
:1021B000120202430A6004339BB2B7E7012AB5D189
:1021C0000A4A521AE15C1160F5E7084959180A6099
:1021D0000433ACE7000004403C00044038000440F5
:1021E00034000440300004400C000440000104406E
:1021F000040004401000044014000440F7B515002A
:1022000080221C001023D2050091916807000B4327
:1022100093600023654AD730136001F0FDFD9D23D4
:102220003E009B00F9583B00CA363200FC330029BF
:1022300000D07FE0586801F0BFFC390032785C4B79
:10224000CB311A604B780A781B0213438A78AC466C
:1022500012041A43CB78281D1B061343554A1BBA98
:1022600013604B790A791B0213438A7912041A43CB
:10227000CB791B061343504A1BBA13604B7A0A7A78
:102280001B0213438A7A12041A43CB7A21001B06DD
:1022900013434A4A1BBA1360009A2B021343484A5D
:1022A00013602200474B1B1B0093009BCE785B18EA
:1022B00001938B7836061B0433430E78043833437E
:1022C0004E78043136023343019E33600328ECDC40
:1022D0000321A808431C9B002940800003292BD11F
:1022E0003849E5185E18A9786D78E35C09042D0279
:1022F000294319433160030008330021FF2B2DDDF2
:10230000314B324919600F21314B196001232749A4
:102310000B60304B19680029FCD006211B680B406C
:10232000042B20D080220020D20593680A318B43F1
:102330009360FEBD01217DE7022908D121495D1886
:10234000E1184978E35C090219432960D3E70129C0
:10235000D3D11C495918E35C0B60CCE71948181815
:1023600001600433CAE7002310490B606346002B69
:102370000CDC3B00FC335A68102101325A60802289
:10238000D205936801208B439360D2E7009B9B1892
:102390001B68190A13705170190C1B0ED37004239B
:1023A0005B4291709C440432E0E7C0460000044068
:1023B0003C00044038000440340004403000044035
:1023C0000C0004400001044004000440080F000019
:1023D000100004401400044070B5061E19D00222FB
:1023E0005A4B9B799343012B13D1594B1A78FF2AEF
:1023F0000FD15A78FF2A0CD19A78FF2A09D1DA78BE
:10240000FF2A06D11A79FF2A03D15B79FF2B00D16D
:1024100099E0504B0C201A78012A08D000224E4D2A
:102420001A7029780B00093B042B01D8212070BDBC
:102430004B1F012BFAD9454CA37B042B00D982E01A
:10244000A279032A00D97EE09A1ED2B2012A02D8CC
:1024500060881F2877D9002E56D0012E73D1A0880E
:102460000128E3D0002907D1581E032803D801F022
:1024700055FB121715122E702978481E032811D803
:102480000025364B1D602823237501F0C5FDA842A9
:1024900027D0A580CAE702212970EDE70421FBE7D8
:1024A0000321F9E707390129C0D82D490968C96A0C
:1024B0008906BBD52B4908780028B7D1012A01D954
:1024C000002BB3D102230B708021274D26338901C5
:1024D0002878237501F090FC80212878890101F08B
:1024E0008BFD0123A380214B1B78002B0AD0FA22FD
:1024F00080211F4B92001B8809025A431A4B1878FF
:1025000001F0AAFB002092E701F086FB2B78A68061
:10251000073B012B03D917482E7001F01DFD114B0D
:10252000114C1A78002A06D08021002220788901D7
:102530001A7001F061FC01F0CFFC802120780902C3
:1025400001F05AFCDEE7122071E7C046A60BFF1F20
:102550006B09FF1F1A09FF1F1C09FF1F4809FF1FF6
:102560004464FF1F2309FF1F1B09FF1F2109FF1FD1
:102570002C09FF1F0010004010B5002901D001F008
:102580002BFB10BDF7B5604B01919978A1239B00FF
:102590004B435E4A060014681022E418D6235B0001
:1025A000E0583623FF33E35C00279343222B41D1CD
:1025B000574B0F3A1A600760012501F0B5FC019BEB
:1025C0001880E8235B00E35C002B01D0B34258DDA8
:1025D0000023504FFB70AD33FF33E3581A68002AD5
:1025E00003D09B88DB439B071DD03823FF33E35C7C
:1025F000002B18D09B235B00E35C002B13D1D1335D
:10260000FF33E35CB3420EDAA4235B00E15AE01827
:10261000090A023101F010FB23000122FE33013EC2
:1026200001351A87FA70E8235B00E35C002B2AD09F
:10263000A8B2FEBD03683D00002BBED081880430E7
:10264000090A023101F0F8FAD6235B00E3581F6053
:10265000B2E72300B133BA00FF33985801378188BD
:102660000430090A023101F0E7FAE8235B00E35C79
:10267000BB42EEDCE822F61AED1800235200A35408
:10268000A6E70027F1E7200001F0AEFC00281FD0EC
:10269000002E1DDD7319882647190193B60020000E
:1026A00001F012FB5A308000201840680135818803
:1026B0000430090A023101F0BFFA200001F0ECFBFE
:1026C000A3590133A351BD4202D0019B9D42E6D1E3
:1026D000114BE35C002BABD095239B00E35C002BFC
:1026E000A6D00E4BE15A0029A2D00D4AA35C994214
:1026F00002D90133A3549BE700231A212000A354DD
:1027000001F022FA94E7C046300DFF1F3409FF1F85
:1027100000140340E010FF1F5A0200007202000084
:102720005E0200000D4970B54A6E0D4CD2038B69F4
:10273000D20BA24206D80B4D0224AA4204D901F0C2
:10274000D3FB70BD02246442E21815007E242540AC
:102750002242F4D0A3432B438B61F0E700F000400A
:102760000A200000FC1C0000F8B51D4B1D4F1A7814
:10277000002A10D1BA7B002A02D101321A7003E07C
:10278000032AFAD0022AF8D001F046FC00220120E8
:10279000154B1A70F8BD154B154D1C68154B9E78DE
:1027A00001232B702878C0B200F09EFBBB7B002B6E
:1027B0000BD101F0F1FBA1239B007343E4188323A9
:1027C0009B00E41823782B70E4E7032B02D101F07F
:1027D00013FAF0E70020022BDCD101F0ADFBEAE7B1
:1027E0001C09FF1FA60BFF1F2309FF1F3409FF1F32
:1027F000490AFF1F300DFF1FF0B587B00EAD2F78CF
:102800000FAD2D780593AC46634614000E4D0CAA0F
:1028100012782E7803930D9B009201932200059B62
:10282000029701F041FB2E70012C01D0042C08D13D
:10283000802206498B889343054A1278D2011343BC
:102840008B8007B0F0BDC0461C09FF1F6C11FF1F35
:102850007809FF1F0B001B3B70B504003020E02BF4
:102860000DD81300E025493BFF3B9BB2ED00AB4286
:1028700005D8034B200019825A8201F005FA70BD79
:102880008410FF1F10B501F05FFB054B00205B6853
:10289000052B04D9034A5268D20200D4980810BD0F
:1028A00000100040FCE100E070B501F0B5F90D4BFF
:1028B0001B68FC33DC691D6AFFF7E4FF641984427E
:1028C00004D2094B01241B68002B07D004220024EA
:1028D000064B1A70064A93690133936101F0FCFAC2
:1028E000200070BD4464FF1F9809FF1F2309FF1FCC
:1028F000FC0FFF1F70B50C4D2B68FC335C6A01F0B8
:102900008BF9FFF7BFFF2B680025FC339B6AE318A8
:10291000834204D2054B1B68AB4200D1051B01F07A
:10292000DBFA280070BDC0464464FF1F9809FF1FF2
:10293000D722044B92009B5810B5002B00D098472B
:1029400010BDC0460000FF1F10B501F0CFF8FFF723
:10295000EFFF2749274BCA6D274C1A4084235B00A1
:102960001343CB65254B1B68186A01F005FB244B0C
:10297000244A1A60244B254A1A60A022244B520094
:102980001A60244B187801F05FF92000224901F009
:10299000C3FA0023A3600233A360204B20492360C5
:1029A00003232048A36001F0B7FA10221E4BFF203A
:1029B0001A60802252031A60802292031A608022D9
:1029C00012041A6001F0F0FA012001F03DFAFA2039
:1029D000400001F0F9F9582001F046F9134801F0E0
:1029E000C3F9012001F0B8F9072001F01DFB10BD6B
:1029F00000F0004000FEFEFF141000404464FF1F82
:102A0000000003400180063DBC0003403408000084
:102A1000A40003404A0AFF1F71020000C30900001E
:102A2000FFFF3F002810004000E100E0307500008B
:102A3000674E336888331B6883F3088801F0FCF91C
:102A4000644A6549136800200B401360634B644A75
:102A50001B68934200D1A6E001F02EFA0221614AE0
:102A600013688B431360FFF76FFF5F4B5F4C187861
:102A7000C0B201F0B9F80023A3600233A3605C4B3D
:102A80000120236001F078FA0323A36001F0F4F938
:102A9000040001F059FA050001F0EEF9554B1860F9
:102AA00001F052F9544B1968621A531EA14200D228
:102AB00013008022D203934201D39B029B0A326807
:102AC000D16AC90700D471E04C491C0C09689BB25B
:102AD0004C4359432402090A641803264849FC322E
:102AE00093680A6847489B1A474A0768126847492B
:102AF0009B18474A9A1833409208DB190A60036012
:102B0000042B03D9013233400A6003600E68414947
:102B1000A619300001F078F93F4F3E493B68C318D1
:102B20003B603000019301F087FA3C4E3068081892
:102B300038493060884205D9019B01333B6001F080
:102B40007BFA316001F030F8354B1B78002B0DD04B
:102B500001F0FAF9334B621B196812188A4232D21B
:102B60004919091B091A304801F0D6F92F4E337A5A
:102B7000002B0ED001F0E8F9621BF16812189142A7
:102B800024D94919091B091A294801F0C5F900235C
:102B90003372284B83F3088801F086F8002001F097
:102BA0008BF901F0E9F801F087F95CE7DC019900A5
:102BB0000234641A5900641A09214B438033CB4014
:102BC000A408E41889E7FA218900CCE71A49DBE771
:102BD0004464FF1F1CF00040FFFFC1FF0C0AFF1FF1
:102BE000B641210310000040490AFF1F14100040A5
:102BF000C3090000100AFF1F340AFF1F380AFF1F15
:102C0000200AFF1F280AFF1F1C0AFF1F240AFF1F9C
:102C1000C4090000710200006008FF1F2C0AFF1F9A
:102C20001C09FF1FE408FF1F00100040740BFF1F6A
:102C30003C10004000000020DC050000A022054BF5
:102C400092009B5810B5002B01D0984710BD01F0A1
:102C500003F9FBE70000FF1FA122054B92009B58E0
:102C600010B5002B01D0984710BD01F0F5F8FBE737
:102C70000000FF1FA222054B92009B5810B5002BAD
:102C800001D0984710BD01F0E7F8FBE70000FF1FF7
:102C9000A322054B92009B5810B5002B01D09847FA
:102CA00010BD01F0D9F8FBE70000FF1FA422054B7F
:102CB00092009B5810B5002B01D0984710BD01F031
:102CC000CBF8FBE70000FF1F70B501F03DF94F4B5B
:102CD000186000F079FF0400C30702D400F0ECFF95
:102CE00070BD00224A4B1A604A4B187801380428FC
:102CF00029D800F013FF0320181C2400200001F045
:102D00005BF90128ECD0444C2378042B6ED100F001
:102D1000B3FF0028E4D000F087FF582000F0A4FFA4
:102D200002232370DCE7200001F06EF9E9E72000C0
:102D300001F0E2F8E5E7200000F0D6FFE1E720002F
:102D400001F02AF8DDE700F017FF0500012808D19F
:102D5000324B1B78053B012B03D82000FFF76EFF99
:102D6000D1E72D4B1B78022B01D0052B20D1022D52
:102D700028D12B4B9B7BAB431CD12000FFF76CFF72
:102D8000264B18780128BED16405BCD424492522DD
:102D90004B7B034205D1233A13405A425341263319
:102DA0001A000B7D9342AED9322001F0DDF8AAE77C
:102DB000022D07D1194B1B78052B11D12000FFF7ED
:102DC00059FFDDE7012D0BD1012B03D12000FFF7C7
:102DD0005FFF98E7062B03D12000FFF767FF92E71C
:102DE000200001F039F8022D8DD1C9E7032B04D161
:102DF0000C4B987C00F0A0FF72E7072B00D06FE728
:102E0000094B987B00F000FF6AE7C0469C09FF1F52
:102E10009809FF1F9009FF1F2309FF1F1C09FF1FAF
:102E2000A60BFF1FBC0BFF1FD40BFF1FFA210A4B81
:102E30000A4A49001A640A4A5A500A4A04395A503E
:102E4000094A08319A64094A5A50094A5C315A5071
:102E5000084ADA667047C0460000FF1FF927FF1FC7
:102E6000F528FF1FA928FF1FD923FF1F6927FF1F70
:102E7000791EFF1F4D1EFF1FF7B50B0CFF27012208
:102E8000009300233C001E001D009446019089B26F
:102E900062469A401000084018413618B6B2FF2F1B
:102EA00002D1012E00D19FB2009802401A41AD1804
:102EB000ADB2FF2C02D1012D00D19CB20133102BF9
:102EC000E6D10320012E07D1012D04D1019B24015D
:102ED000E4191C700138FEBD102EFCD10238102DF3
:102EE000F9D00230F7E700008023F7B59C46264B67
:102EF000264F01932649274A274D284C284B022864
:102F00001AD1604638600868264E30408026360365
:102F10003043086001990978002909D11660224AD6
:102F20002A60224A2260E02219689143A03A1BE0FD
:102F30008021C9021160F2E766463E600F68194EB3
:102F40003E408027FF023E430E6001990978002928
:102F50000DD1176001280ED1154A2A60154A22604A
:102F6000E02219689143C03A0A431A60F7BD8021F4
:102F700089021160EEE7E0210F4A02432A600F4AFE
:102F800022601A688A43F0E74B0AFF1FE000034003
:102F9000D80003409000034000000340500003406D
:102FA00040000340FFFFE3FF0280063D804508220A
:102FB0000180063D80660822008006988055082220
:102FC000F8B51E4B80261A680020140034403242A7
:102FD00032D11A681A4F32431A6001223B68063018
:102FE00093433B6000F0C8FF0122164D2B681E433F
:102FF0002E603B680A2613433B608027BF00124BBC
:103000001B683B4211D1013EF6B2FF2E09D17E2250
:103010000E4B1C682B68E40B1440934323432B6036
:1030200005E0082000F0A8FFE9E7002EEFD180229C
:103030002B68600893432B60F8BDC046C4F0004085
:103040005CF0004018F0004068F0004060F0004084
:1030500010B500F019FF01215820034A00F064FE6A
:10306000FFF7AEFF10BDC046600AFF1F10B5782203
:103070000021034800F030FE00F096FE002010BD55
:103080003867FF1F70B5040000F0C6FD00230C2058
:103090000B4A010059438D18515C00290DD0A14203
:1030A00008D1012300246B7000F05EFD00F014FFD6
:1030B000200070BD01330A2BEBD11224F6E7C04685
:1030C0003867FF1F70B5040000F0A6FD002319004B
:1030D0001D000D4A1078002806D0A0420CD1557072
:1030E00001310C320A29F5D1002B0AD100F05CFE27
:1030F00000F0F2FE002070BD5078461EB0411B1853
:10310000EEE700F031FDF3E73867FF1FF7B5040085
:103110000C20002384460E4D019267465F43E85D14
:103120007E19A04212D000280BD10A4B9C46624661
:103130001B7808331370019B70707C557160B3600D
:10314000FEBD01330A2BE8D10320F9E70720F7E79A
:103150003867FF1F3467FF1F8020F8B5484BC00554
:103160001B68C1248360474BFF251A680123134362
:103170004361454BA4001A68444B40211A60444BFC
:103180001A68444B1A60444B1A59AA431A51C52273
:1031900092009E58AE433143802699509F583F4934
:1031A000F6010F403E439E509E5880273602360A55
:1031B0003043985080201A5900020A4002431A51A5
:1031C00004341A59364E3F04324080263A431A518D
:1031D0001A5936061202120A32431A5108341A5981
:1031E00080260A4002431A51C32292009F58B446D7
:1031F000AF4337439F509F58294E0F4007439F507E
:103200009F58374080263604374380269F509F586A
:1032100036063F023F0A37439F50C0221F59AF4333
:103220003A431A511A591202120A1643C6221E5163
:1032300092009C58AC4365462C439C509C580025FA
:103240000C4020439850C72080001A58154C11405C
:10325000C02212020A431A50134B1B78DB08AB4200
:1032600001DC0020F8BD2378002B06D0A368002BDA
:1032700000D0984701350C34EEE71220F2E7C04643
:103280004C43FF1F4843FF1FB0F000403067FF1F53
:10329000B4F000402C67FF1F00E100E0FF00FFFFDB
:1032A000FFFF00FF3867FF1F3467FF1F030010B5E3
:1032B0001F2809D8072200201340072404490A7850
:1032C000A24313430B7010BD00230620F5E7C04650
:1032D0003467FF1F054B06491B780A6805485B07E2
:1032E00002401B0B134300200B6070473467FF1F25
:1032F0001CF00040FFFFC1FF70B50C25FFF7EAFF8F
:103300000A4B1C780A4BE4086543ED18002C01D1E8
:10331000200070BD2B78002B06D06B68002B00D0EE
:103320009847013C0C3DF1E71220F2E73467FF1F9C
:103330002C67FF1F1FB5002102220B000191009195
:10334000052000F0A9FC02230B490A681A42FCD1AF
:1033500020230393039B5A1E0392002BFAD1074AA2
:103360001368002BFCDA0B246C442000012100F0D0
:1033700013FC207804B010BD90C8004000C8004085
:1033800013B504000A4B0193019B002B01D11120BE
:1033900016BDFFF7CFFF23000340044205D00520F0
:1033A00000F0EAFD019B013BEDE71800F0E7C046A5
:1033B000FFFFFF0707B500F02FFC80220821D20590
:1033C000936A0191002B01D10739916202210C4AC5
:1033D00011600199481E01900029FAD10331116052
:1033E000053101910199481E01900029FAD111601F
:1033F000002B02D18022D205936200F06DFD07BD43
:1034000000C00040F0B52D4C89B02378002B4FD17F
:10341000FEF7D2FA02232A4F03903A681A42FCD1EF
:1034200020230693069B5A1E0692002BFAD1254EA6
:103430003368002BFCDA0120FFF7A2FF011E02D047
:10344000112009B0F0BD030003220190009005ADEA
:103450009F2000F021FC0321280000F09DFB0223A7
:103460003A681A42FCD120230793079B5A1E079201
:10347000002BFAD13368002BFCDA0120FFF780FF24
:103480000028DDD10398FEF7ABFAAA786B78110417
:103490001B020B4329780B4363601300113B0A495D
:1034A000052B07D801239340A3600B6001232370F1
:1034B0000020C6E780231B03F6E7C0463443FF1F06
:1034C00090C8004000C800409808FF1F1E4B30B550
:1034D0005A6818781D4B85B0D31859424B410121C9
:1034E0000093002300F010FD194B1A4A02259A633D
:1034F00000221A6510325A658022C4219D65164B40
:103500001648D202DA6789004258154B80241A40C7
:1035100080231B0413434350642341200393E40599
:1035200000F006FA402000F003FA6562039D6B1E6E
:103530000393002DFAD103236362FFF73BFFA562DB
:10354000FFF760FF05B030BD4043FF1F95FFFEF75A
:1035500000C80040050001FF04E100E000E100E0D8
:10356000FFFF00FFF0B585B00700FEF725FA022344
:1035700005002D4C22681A42FCD120230093009BA9
:103580005A1E0092002BFAD1284E3368002BFCDA29
:103590000120FFF7F5FE002803D01124200005B01C
:1035A000F0BD234B2360022322681A42FCD1202362
:1035B0000193019B5A1E0192002BFAD13368002B14
:1035C000FCDA0120FFF7DCFE0028E6D1194B1F6072
:1035D000022322681A42FCD120230293029B5A1E26
:1035E0000292002BFAD13368002BFCDA0120FFF79E
:1035F000C7FE0028D1D1104B2360022322681A4253
:10360000FCD120230393039B5A1E0392002BFAD173
:103610003368002BFCDA0120FFF7B2FE041EBCD198
:103620002800FEF7DDF9B9E790C8004000C8004067
:1036300001000006A8C800400180000110B500206C
:10364000FFF790FF10BD000010B5064B18705960D1
:10365000FFF73CFF00211320034AFFF757FD00202E
:1036600010BDC0464043FF1FCD34FF1FF0B504001E
:1036700085B003920291FEF79FF9882263035B0BEA
:1036800052051A438023DB059D6A8023274F009251
:10369000BA68002601901B039A420CD9F823260031
:1036A0001B041E401C4206D08022214B52025E6247
:1036B00019680A431A60002D0BD100F0ADFA0222FE
:1036C0001C4B1A608023DB055A62013A9A6200F0B3
:1036D00003FC0023039A934220D1002D0AD100F06D
:1036E0009BFA144B03221D608023DB055A629D6206
:1036F00000F0F2FB8023BA681B039A4208D9002E1F
:1037000006D000220A4B0C495A621A680A401A6015
:103710000198FEF765F9002005B0F0BD009A029906
:10372000D2181278CA540133D4E7C0463443FF1F7D
:1037300000C8004000C00040FFFFFEFFF0B587B0AA
:10374000029103920400FEF737F9019000F064FA49
:10375000802302250122234EDB0535605D629A62DB
:1037600000F0BAFB204F3B682B42FCD1202304938E
:10377000049B5A1E0492002BFAD11C4D2B68002B7F
:10378000FCDA0120FFF7FCFD002802D0112007B071
:10379000F0BD2000039A029900F0DEF90223040034
:1037A0003A681A42FCD120230593059B5A1E0592C4
:1037B000002BFAD12B68002BFCDA0120FFF7E0FD8B
:1037C000051EE3D100F028FA80230322DB053560D3
:1037D0005A629D6200F080FB0198FEF701F9E0B2A9
:1037E000D5E7C04600C0004090C8004000C8004077
:1037F000F0B5802489B00600FEF7DEF8E405A36A80
:1038000002250393029000F007FA0123304F3D6038
:103810006562A36200F060FB2E4C23682B42FCD152
:1038200020230593059B5A1E0592002BFAD12A4DA1
:103830002B68002BFCDA0120FFF7A2FD002803D043
:103840001124200009B0F0BD244B2360022322681C
:103850001A42FCD120230693069B5A1E0692002B87
:10386000FAD12B68002BFCDA0120FFF789FD021E3C
:10387000E6D11B4B03211E60030001900090202025
:1038800000F00AFA022322681A42FCD1202307938F
:10389000079B5A1E0792002BFAD12B68002BFCDAEB
:1038A0000320FFF76DFD041ECAD100F0B5F9802397
:1038B0000322DB053C605A629C6200F00DFB039B17
:1038C000002B01D1FFF776FD0298FEF789F8B8E7E3
:1038D00000C0004090C8004000C800400100000641
:1038E00094C8004007B5000201910422000A01A912
:1038F000FFF724FF0EBD000073B5050005240B4A39
:10390000A3005B429B1819686B46DE1D3000FFF771
:10391000B3FA022804D133782B55013CEFD276BD9F
:10392000052CFCD00128FAD10230F8E71409001167
:103930001F2807D8012380228340D20591680B43BA
:10394000936070473F2808D80123802220388340A5
:10395000D20551690B435361F3E75F28F1D8012386
:10396000802240388340D205116A0B431362E8E796
:103970001F2807D8012280218240C9058B68934304
:103980008B6070473F2808D8012280212038824070
:10399000C9054B6993434B61F3E75F28F1D80122D6
:1039A000802140388240C9050B6A93430B62E8E7E7
:1039B0001F2810D880230200DB05153A1968012A58
:1039C00006D820229143196019680A431A6070478B
:1039D00001228240F6E73F2811D880230200DB0550
:1039E000353AD968032A06D810229143D960D9689C
:1039F0000A43DA60EBE7012220388240F5E75F28CE
:103A0000E5D842238022181A413B8340D205516AEF
:103A100099435162516A0B435362D8E710B50400D1
:103A2000012813D1A022184992050B685B015B099C
:103A300013430B60154B164A19681140154A0A4387
:103A40001A60402219680A431A6010BD0028FCD190
:103A500001000A2000F058F921000B2000F054F971
:103A6000C0220A4B920019680A4340211A601A6862
:103A70008A431A60B022044912060B685B015B0995
:103A800013430B60E1E7C04614F000401CF0004017
:103A90007F00FEFF80FD010072B6074A1368013304
:103AA00013600422054B1A600023054A136080222C
:103AB000D2055360FEE7C0467808FF1FC0F0004003
:103AC000C4F0004005490B68002B05D1044A0A6088
:103AD00004490A60044A13607047C046140AFF1F75
:103AE000841E0000380AFF1FC4F000400023034A70
:103AF0001360034A1360034A1360704754F0004098
:103B000040F1004044F1004002B4714649084900C8
:103B1000095649008E4402BC7047C04602B4714643
:103B200049084900095C49008E4402BC7047C04600
:103B300003B47146490840004900095A49008E44BF
:103B400003BC70470000000001B40248844601BC79
:103B5000604700BF53B9000001B40248844601BC6D
:103B6000604700BF9573010001B40248844601BC60
:103B7000604700BF21A9000001B40248844601BC8F
:103B8000604700BFDD0C010001B40248844601BC5F
:103B9000604700BFE94C010001B40248844601BC03
:103BA000604700BF3D71010001B40248844601BC7A
:103BB000604700BFD544010001B40248844601BCFF
:103BC000604700BF2144000001B40248844601BCA4
:103BD000604700BFBD0B010001B40248844601BC30
:103BE000604700BFE9D4000001B40248844601BC2C
:103BF000604700BF8914010001B40248844601BC3B
:103C0000604700BF75F8000001B40248844601BC5B
:103C1000604700BFC1F7000001B40248844601BC00
:103C2000604700BF75A9000001B40248844601BC8A
:103C3000604700BF6DF6000001B40248844601BC35
:103C4000604700BFC115010001B40248844601BCB1
:103C5000604700BFEDA5000001B40248844601BCE6
:103C6000604700BF8B52010001B40248844601BC8A
:103C7000604700BF7912010001B40248844601BCCC
:103C8000604700BF01D7000001B40248844601BC70
:103C9000604700BF116E000001B40248844601BCB9
:103CA000604700BF496D010001B40248844601BC71
:103CB000604700BF7997000001B40248844601BC08
:103CC000604700BFDD0A010001B40248844601BC20
:103CD000604700BFD9B0000001B40248844601BC6F
:103CE000604700BFB70E000001B40248844601BC23
:103CF000604700BFF535010001B40248844601BCAD
:103D0000604700BFBD5C010001B40248844601BCAD
:103D1000604700BF99A2001101B40248844601BC6B
:103D2000604700BFE90B010001B40248844601BCB2
:103D3000604700BF0167010001B40248844601BC2E
:103D4000604700BF4DF9000001B40248844601BC41
:103D5000604700BFC166010001B40248844601BC4F
:103D6000604700BFE512010001B40248844601BC6F
:103D7000604700BF8D11010001B40248844601BCB8
:103D8000604700BF8552010001B40248844601BC6F
:103D9000604700BF51B8000001B40248844601BC2E
:103DA000604700BFF935010001B40248844601BCF8
:103DB000604700BFADAE000001B40248844601BCBC
:103DC000604700BF8937010001B40248844601BC46
:103DD000604700BF8512010001B40248844601BC5F
:103DE000604700BF41B6001101B40248844601BCDF
:103DF000604700BF8D82000001B40248844601BCC8
:103E0000604700BFB352010001B40248844601BCC0
:103E1000604700BF090E000001B40248844601BC9F
:103E2000604700BF8944000001B40248844601BCD9
:103E3000604700BFF9ED000001B40248844601BCB0
:103E4000604700BFC9A9000001B40248844601BC14
:103E5000604700BF6911010001B40248844601BCFB
:103E6000604700BFE917010001B40248844601BC65
:103E7000604700BFDD3F000001B40248844601BC3A
:103E8000604700BF156B010001B40248844601BCC5
:103E9000604700BFED68010001B40248844601BCE0
:103EA000604700BF5976010001B40248844601BC56
:103EB000604700BF9D6A000001B40248844601BC0F
:103EC000604700BF016C010001B40248844601BC98
:103ED000604700BFE927000001B40248844601BCE6
:103EE000604700BF9DA9000001B40248844601BCA0
:103EF000604700BFD1AE000001B40248844601BC57
:103F0000604700BF0534010001B40248844601BC8B
:103F1000604700BFC56D010001B40248844601BC82
:103F2000604700BF2D6C010001B40248844601BC0B
:103F3000604700BFCD0C010001B40248844601BCBB
:103F4000604700BF19FA000001B40248844601BC72
:103F5000604700BFC95C010001B40248844601BC4F
:103F6000604700BFC1A5000001B40248844601BCFF
:103F7000604700BF6137010001B40248844601BCBC
:103F8000604700BF0189000001B40248844601BCBB
:103F9000604700BFCD4C010001B40248844601BC1B
:103FA000604700BFE9F6000001B40248844601BC46
:103FB000604700BFED6B010001B40248844601BCBC
:103FC000604700BF0134010001B40248844601BCCF
:103FD000604700BF85C1000001B40248844601BCAF
:103FE000604700BF6D0B010001B40248844601BC6C
:103FF000604700BF71B0000001B40248844601BCB4
:10400000604700BF0D52010001B40248844601BC64
:10401000604700BF0934010001B40248844601BC76
:10402000604700BFA9D8000001B40248844601BC23
:10403000604700BFF90D010001B40248844601BC8D
:08404000604700BF090E0000FB
:1040480002000000F6BE001101000000F8BC0011DB
:1040580002000000F2BE0011010000008840FF1FAE
:104068000200000000BD001101000000C861FF1F30
:1040780002000000F0BE0011030000003C61FF1FB9
:104088001200000002000000F6BE0011010000004E
:1040980040BD001102000000F2BE00110100000046
:1040A8003DBD0011020000004ABD001103000000E0
:1040B8007761FF1F02000000F0BE0011030000003E
:1040C8008C61FF1F02000000F2BE00110100000019
:1040D8003CBD00110200000048BD001103000000B3
:1040E8004D61FF1F02000000F0BE00110300000038
:1040F8006E61FF1F02000000F6BE00110100000003
:1041080084BD001102000000F2BE00110100000091
:10411800D141FF1F0200000096BD00110100000000
:104128007BBD001102000000F2BE0011010000007A
:10413800D041FF1F0200000094BD001101000000E3
:104148009461FF1F02000000F2BE00110100000090
:10415800CF41FF1F0200000092BD001101000000C6
:104168006BBD001102000000F2BE0011010000004A
:10417800CE41FF1F0200000090BD001101000000A9
:1041880066BD001102000000F2BE0011010000002F
:10419800CD41FF1F020000008EBD0011010000008C
:1041A80061BD001102000000F2BE00110100000014
:1041B800CC41FF1F020000008CBD0011010000006F
:1041C8005CBD0011020202020202000000000000B1
:1041D80016150000B14B0011774B0011E4BD00111A
:1041E80090011D0018001800FFFF070102030405D5
:1041F80006020106000000000000000000000000A8
:1042080000000000000000000000000000000000A6
:104218000300000002000000F6BE001101000000CB
:1042280004BE001102000000F2BE001101000000EF
:104238008C42FF1F020000000EBE001101000000AA
:10424800C261FF1F02000000F0BE00110300000061
:104258002C64FF1F02000000F2BE001101000000E4
:104268008C42FF1F020000000CBE0011010000007C
:10427800C461FF1F02000000F0BE0011030000002F
:104288002464FF1F120800000000000000C6C600DA
:1042980000000000000000001311000000010000F1
:1042A80000000111FFFF00005048593600000000CF
:1042B800000000000B000500F0000000B40000281A
:1042C800002800283075A000A000A000A000000869
:1042D8000008E001F00010001000100010001000AD
:1042E800100050005000500010001000D0070000CF
:1042F800000000000F0001000500307507001000E5
:10430800010081FF00000000FF000000817400111F
:104318008972001119700011FFFF0100FF000000F1
:104328009D9E0011199C0011319B00110000000096
:104338000000000000000800040000003B00010825
:104348005902E00188212800FF0000000200000057
:10435800F6BE001101000000BCBF00110200000001
:10436800F2BE001101000000D143FF1F020000004F
:10437800EEBE001101000000F067FF1F0200000000
:10438800F2BE001101000000D043FF1F0200000030
:10439800ECBE001101000000CE43FF1F0200000028
:1043A800F2BE001101000000CC43FF1F0200000014
:1043B800EABE001101000000C443FF1F18001800E6
:1043C8001D0090010200000302020000020000002C
:1043D800F6BE001101000000D0BF0011020000006D
:1043E800F2BE0011010000001444FF1F020000008B
:1043F800E8BE0011000000000000000002000000FC
:0E440800F0BE0011030000001068FF1F20FF2F
:040000051FFF184180
:00000001FF
